:020000040800F2
:10000000E0100020050100083F38000831290008F1
:100010003D380008450F00084D6100080000000051
:100020000000000000000000000000008147000800
:10003000EF1A0008000000009D3D0008694A000812
:100040001F0100089D3B00081F0100081F01000858
:100050001F0100081F0100081F0100081F01000800
:100060001F0100081F0100081F0100081F010008F0
:100070001F0100081F010008B11500081F0100083A
:100080001F0100081F010008410700081F010008A8
:100090001F0100081F0100081F0100081F010008C0
:1000A000D94A0008B94B00081F0100081F010008C9
:1000B000BD4B0008AD4E0008095100081F010008A3
:1000C0001F0100081F0100081F0100081F01000890
:1000D0001F010008455C00081F0100081F010008FF
:1000E0001F0100081F0100081F010008DFF810D0E1
:1000F00000F0E8FA0048004729720008AFF30080DA
:10010000E01000200648804706480047FEE7FEE76B
:10011000FEE7FEE7FEE7FEE7FEE7FEE7FEE7FEE7B7
:10012000894A0008ED0000082DE9F0410024061B73
:10013000254671F1000605DA01240027D0EB0700FF
:1001400067EB0101161E73F1000605DA0027D2EBFA
:100150000702012567EB030300F0D0F986460E463F
:1001600017469C46AC4204D00025D0EB050E65EB4B
:10017000010624B10020D2EB000760EB030C7046AF
:1001800031463A466346BDE8F08140EA01039B07E9
:1001900003D009E008C9121F08C0042AFAD203E0FC
:1001A00011F8013B00F8013B521EF9D2704780EA7A
:1001B000010210B502F00043400022D04A001FD0D7
:1001C000010E01EB1261C0F35600C2F3560240F477
:1001D000000042F40002A0FB022000047F39140456
:1001E00000D0401C50EA124001D44000491EC2B267
:1001F0000C0604EBD010401C4008802A02D003E01B
:10020000002010BD20F00100002900DA0020184372
:1002100010BD2DE9FE4F81EA030404F0004421F0F3
:10022000004100944FF0000B23F0004350EA01041A
:100230005ED052EA03045BD0C3F30A54C1F30A55FB
:100240002C44A4F2F3340194A0FB0254C1F3130133
:1002500041F48011C3F3130343F4801301FB024400
:1002600000FB034E840A970A44EA815447EA835705
:10027000A4FB076802958D0A05FB07854FEA932CBE
:1002800004FB0C542705029D4FEA065847EA16372F
:10029000B5EB08056EEB070C870E920E47EA811747
:1002A00042EA8312A7FB0201B6EB0B0164EB0004E8
:1002B0002B0D43EA0C335E1844EB1C50DA465146D2
:1002C000E7FB0201C5F313044FEA0B3343EA14536F
:1002D0004FEA0432019C43EA0603A4F10C040294A1
:1002E000009CCDE900B400F09FF903B0BDE8F08FA9
:1002F00000200146F9E72DE9F04D81EA030404F0FE
:10030000004B21F0004514464FF0000A23F0004155
:1003100050EA050220D054EA01021DD0C5F30A5765
:100320000246C5F31303C1F31300C1F30A5640F4A8
:10033000801543F48013A7EB0608101BD64608F27D
:10034000FD3873EB050002D308F1010801E09218B3
:100350005B41B8F1000F03DA00200146BDE8F08DE3
:1003600000204FF48011064684460EE0171B73EB05
:10037000050705D3121B63EB050306434CEA010C8A
:1003800049084FEA300092185B4150EA0107EDD16D
:1003900052EA030012D082EA040083EA050108430E
:1003A00005D0101BAB4106D20122002306E000223B
:1003B0004FF0004302E06FF0010253101AEB060009
:1003C0004CEB085110EB0A0041EB0B01BDE8F04D7E
:1003D00000F01BB970B521F0004303430CD0C1F30A
:1003E0000A550024D5EB040564EB0403D617AD1AB7
:1003F000B34102DB0020014670BD201841EB0251E1
:1004000070BDC10F80EAE0700844CA07962300213E
:1004100000F0CDB896230022114600F0C8B80EB502
:10042000C10F80EAE0700844CA07002140F233435C
:100430008DE80E000A460B4600F0F6F803B000BD4A
:100440000EB540F2334102910021CDE900110A4678
:100450000B4600F0E9F803B000BD00F0004220F0C8
:100460000040C10DC0F3160040F400007F2901DAFE
:1004700000207047962903DCC1F19601C84001E0D5
:1004800096398840002AF4D04042704770B5C1F3D5
:100490000A5201F000450024C1F3130140F2FF337A
:1004A00041F480119A4201DA002070BD40F23343DA
:1004B0009A42A2F2334203DC524200F05FF800E0BD
:1004C00090402C43F1D0404270BDC1F30A5210B5A8
:1004D000C1F3130140F2FF3341F480119A4201DA73
:1004E000002010BD40F233439A42A2F2334203DCB3
:1004F000524200F043F810BD904010BD2DE9F05F6E
:100500000546002092469B46884606468146402482
:100510001BE0284641464746224600F02FF8534646
:100520005A46C01A914110D311461846224600F08F
:1005300016F82D1A67EB01084F46224601200021CC
:1005400000F00DF817EB00094E41201EA4F1010444
:10055000DFDC484631462A464346BDE8F09F202A64
:1005600004DB203A00FA02F1002070479140C2F10A
:10057000200320FA03F3194390407047202A04DB3C
:10058000203A21FA02F00021704721FA02F3D0400C
:10059000C2F1200291400843194670470029A8BFC4
:1005A0007047401C490008BF20F00100704710B49C
:1005B000B0FA80FC00FA0CF050EA010404BF10BC51
:1005C000704749B1CCF1200421FA04F411FA0CF17E
:1005D00018BF012121430843A3EB0C01CB1D4FEAB7
:1005E00000614FEA102042BF002010BC704700EBB2
:1005F000C35010440029A4BF10BC7047401C4900E0
:1006000008BF20F0010010BC704710B5141E73F134
:10061000000408DA401C41F1000192185B411A43C2
:1006200001D120F0010010BD2DE9F04D92469B460E
:1006300011B1B1FA81F202E0B0FA80F220329046B4
:10064000FFF78DFF04460F4640EA0A0041EA0B011E
:1006500053465A46084313D0114653EA010019D0B5
:10066000C8F140025046FFF789FF05460E46504646
:1006700059464246FFF773FF084305D0012004E0C6
:1006800020463946BDE8F08D0020054346EAE07675
:100690002C4337430A986305E40AA0EB08000022C4
:1006A000FD0A44EA47540A3002D500200146E9E732
:1006B000010510196941DDE9084500196941BDE8E6
:1006C000F04DA2E7064C074D06E0E06840F001035C
:1006D00094E8070098471034AC42F6D3FFF70AFDC0
:1006E000F09300081094000870B58C1810F8015BA6
:1006F00015F0070301D110F8013B2A1106D110F8BB
:10070000012B03E010F8016B01F8016B5B1EF9D1BE
:100710002B0705D40023521E0DD401F8013BFAE744
:1007200010F8013BCB1A921C03E013F8015B01F8AF
:10073000015B521EF9D5A142D8D3002070BD000044
:1007400070B54F4C4FF490652946204600F01BFAD7
:10075000002866D02946204600F0A8F849490888B4
:10076000401C08800121204600F0ECFA464942F284
:100770001072B1F85000904202D2401CA1F8500013
:1007800006F02EFF05F056F8404DB5F91410B5F9F6
:10079000120005F01DFE3E4CA5F84E002080A16819
:1007A00020468847A088A5F8500003F0B1F807F06C
:1007B00019F8384E384C3078082833D045F6AC302C
:1007C000606042F6EF60A06042F2C400E06033482F
:1007D000008A2080208E6080A16B2F488847208E61
:1007E00069882F4C08444FF6FF7101EA8000688643
:1007F000207A4FF0000540071DD501F007FB29497D
:1008000049F6A2400880284840F21A62C188491C73
:1008100089B2C180914204D3A16821F00401A16092
:10082000C58070BD41F2130060604FF48060A0602D
:1008300040F61B50CAE730780A281BD2DFE800F0E8
:100840001A0616050A050D1A1114EAE7BDE87040EC
:1008500005F062BF07F0E0FE08E0BDE8704002F07E
:10086000A1BD06F0D3FA01E007F014F9BDE870402D
:1008700007F010B900F0FEFB84F8B65070BD000020
:1008800000240140F80600203C0100206000002008
:1008900014070020EF060020D0000020EC0100200B
:1008A00098020020442C0140200900206FEA112109
:1008B000016070470029816802D041F0010101E028
:1008C00021F00101816070470029816802D041F464
:1008D000807101E021F48071816070472DE9F04161
:1008E000824E92B0304600F00BF90BA800F039FAB6
:1008F00001214FF4C06003F007FB00248DF8314064
:100900004FF46020CDE90D044FF4A0204FF009080A
:100910000B9001278DF83C808DF830700BA9304684
:1009200000F080F9724D8DF831408DF830708DF8FF
:100930003C700BA9284600F075F901231A460F21D7
:10094000304600F0C0F9022201231146304600F083
:10095000BAF9012303220021304600F0B4F9012343
:1009600004221946304600F0AEF9012305220B217E
:10097000304600F0A8F9012306220421304600F099
:10098000A2F9012307220821304600F09CF9012337
:1009900008220321304600F096F9012309220A219A
:1009A000304600F090F90121304600F084F9012131
:1009B000284600F080F901231A460521304600F050
:1009C00055F901231A460621284600F04FF9002167
:1009D000304600F0CBF84FF4E041284600F0C6F86E
:1009E0000121304600F0B8F80121284600F0B4F8A3
:1009F0000121304600F0A6F80121284600F0A2F8B7
:100A00000121304600F09EF90121284600F09AF9B4
:100A100040F61451374804F04EFE12208DF8400085
:100A200002208DF841008DF842408DF8437010A8E7
:100A300002F032FF01224FF49061304600F0E8F8F6
:100A400001213046FFF740FF01213046FFF732FF1A
:100A500001212846FFF72EFF304600F06EF93046A0
:100A600000F09FF80028FAD1304600F075F93046C2
:100A700000F082F80028FAD1284600F05EF92846F6
:100A800000F08FF80028FAD1284600F065F92846D2
:100A900000F072F80028FAD10121084603F010FA9C
:100AA000154D284600F0C0FD684600F068FE0F486E
:100AB00001A94C300090114881E811018020CDE956
:100AC00004404000069080000790202008904FF4DA
:100AD0004050CDE909046946284600F033FE012163
:100AE000284600F095FD12B0BDE8F08100240140D9
:100AF00000280140002C014008000240A80200200C
:100B00000D4910B5884202D1012144150AE00B4974
:100B1000884202D10121041504E0094988420AD122
:100B20000121CC03204603F0FBF92046BDE810402C
:100B3000002103F0F5B910BD002401400028014058
:100B4000003C01400029816802D041F4801101E09D
:100B500021F48011816070470029816802D041F43E
:100B6000004101E021F4004181607047826822F475
:100B7000E0420A43826070470146002089684907C5
:100B800000D50120704710B50246002054680B0ABA
:100B9000C9B20C401168194202D0002C00D00120CB
:100BA00010BD014600208968090700D50120704763
:100BB00038B501211C2003F0A7F9FF20ADF8000093
:100BC00000248DF8034003258DF8025069460D4836
:100BD00001F01EFB0120ADF800008DF803408DF8F8
:100BE00002506946084801F013FB2320ADF80000CD
:100BF0008DF803408DF802506946044801F008FB67
:100C000038BD000000080140000C01400010014008
:100C1000002A4268C9B201D00A4300E08A43426018
:100C20007047000010B542680E4B0C791A400B68F3
:100C300042EA04221343436083680B4A1340D1E91C
:100C4000024222434C7943EA44031A438260C26A57
:100C5000097C22F47002491EC9B242EA0151C16204
:100C600010BD0000FFFEF0FFFDF7F1FF70B5072497
:100C700009290AD9C568A1F10A0606EB4606B4405F
:100C8000A543B3401D43C56007E0056901EB41067C
:100C9000B440A543B3401D430561836BC3F30154C6
:100CA000121B921C02EB82041F22A2409343A1401C
:100CB0000B43836370BD826B491E22F4401242EAEB
:100CC00001518163704770B5072409290AD9C568A5
:100CD000A1F10A0606EB4606B440A543B3401D4306
:100CE000C56007E0056901EB4106B440A543B34088
:100CF0001D4305611F23072A09D2446B521E02EBD4
:100D0000820293409C4391400C43446370BD0D2A82
:100D100009D2046BD21F02EB820293409C439140A4
:100D20000C43046370BDC46A0D3A02EB8202934027
:100D30009C4391400C43C46270BD816841F008013E
:100D4000816070470029816802D041F4A00101E070
:100D500021F4A00181607047816841F00401816045
:100D6000704700210160017141718160C160012102
:100D70000174704770B51E4C214694F83800B1F8E4
:100D8000425006281ED9B4F84A10B4F84C00A1EB22
:100D9000000202F10902122A04D8FFF751FB0022D7
:100DA000144B0AE0884204D2FFF74AFB0022124BA0
:100DB00003E0FFF745FB0022104BFFF72AFAFFF78D
:100DC00084FB09E005D12846FFF73AFB0C4A0D4B9E
:100DD000F3E70D4951F82000C5EB45116063B0EB16
:100DE000410F03D9C5EB45104000606370BD0000A2
:100DF0003C04002000003440000033400000354037
:100E00006766666666E64B40988B000810B50C4C2A
:100E10002078400713D5FFF7ADFF0A49A08E088060
:100E200008483038018821F010010180001F018836
:100E300041F010010180207820F00400207010BDE6
:100E40003C04002040040040F0B4184816494FF418
:100E50009677436C08468A68046815485FEAC25C66
:100E600042F00806007822F008054FEA047415D510
:100E7000002C08DB120714D408B1082811D1BB429A
:100E80000FDA8E6007E012070BD508B1082808D1E9
:100E9000BB4206DA8D60F0BC05F0BCBD002CF2DA76
:100EA000E8E7F0BC70470000980200203C010020F9
:100EB000EF06002070B506464089204B204C4FF4C9
:100EC0008071002580B362887AB1012A0CD1E18853
:100ED000491C89B2E1803289914205D36580E58061
:100EE000FF2801D0401E708170BD7088228890421A
:100EF00001D9012200E00022184601F012FA7088A0
:100F0000B18801442088401C80B220808142EBD807
:100F10002580A088401C80B2A080F1888842E3D35D
:100F200001206080A58070BDFFE70022184601F017
:100F3000F8F9A580E58025806580F4E7000C014084
:100F4000AC050020FEE70000FCB505464FF6FF7635
:100F500000200C46ADF8006048F205078DF804004B
:100F600020E000BF15F8010B8DF8040001A9084628
:100F700002F0F6F8BDF800009DF8041080EA0120A8
:100F8000ADF800005FF00000BDF800100A0402D5C3
:100F900087EA410101E006EA4101401CADF800107A
:100FA0000828F1DB641EDDD26946084602F0C2F86B
:100FB000BDF80000FCBD00000246002004E000BFB8
:100FC00012F8013B1844C0B2491EF9D27047000024
:100FD00070B5144A85B01088002413490194009418
:100FE000039420460494138807E00D8B009E35443B
:100FF0000095CD8B019E3544019515889D42F4D016
:10100000401CC0B28028EED30098411107484180AF
:10101000848001984111064881830183818205B053
:1010200070BD0000F806002098020020C6050020D0
:10103000B404002030B50E4902880A800C4A438867
:10104000083A13800B1F808818802024151F2C80DD
:101050000020401C80B27328FBD341F2111008809D
:1010600044F64800108047F2480018802C8030BDBC
:10107000202C0140114944F648000880091D46F61D
:1010800048000880091D41F2111008800B48001F1C
:10109000018841F02001018009480021A0F8641076
:1010A000A0F86210A0F86010A0F85E10A0F85C1024
:1010B000A0F85A100348418181827047182C0140E2
:1010C0009802002060000020F0B54F4B4F480021EF
:1010D000DA7A0778802A27F001057DD31C684C4B0B
:1010E00002F01F0253F822204A4B14421A6802D021
:1010F00042F0200201E022F02002474C1A60474EE5
:1011000094F800C0464CBCF1020FB4F9044043D13E
:10111000B3F808C0CCF3C00ECCF3002CE6453BD0AE
:101120003C4D2C3D95F802C0BCF1000F04D0BCF141
:10113000010F0FD0A97033E05FEA025C30D55FEA9F
:10114000826C2DD44FF0010C85F802C027F0040505
:10115000057025E05FEA025C22D45FEA826C1FD54D
:101160005FEA477C0BD447F004070770B0F802C071
:10117000BCF1000F06D0418027F00107077002275D
:10118000AF700DE04480002CF9DD47F001070770D7
:10119000244FFF6A4761F2E7057041803180418149
:1011A0001C4DC78895F846500FB9002C17DC077BFB
:1011B000AF4214D1B0F9027007F26667BC420EDC90
:1011C000194FBF895FEA477C09D45FEA877C06D460
:1011D0005FEA427C03D500E012E0FF0709D0077800
:1011E0005FEAC77C05D027F0010707704180318096
:1011F0004181C4800573500960F3CB221A60F0BDB1
:10120000057041804181F0BDCC0500200809002017
:10121000F88F000898020020EF060020100100203F
:10122000C605002060000020100A00202DE9F047CC
:1012300096B000240C940D940E940F9472B69048BE
:10124000816941F400718161816941F4806181614A
:101250004FF4004002F02AFE8A4D00212846FFF795
:1012600033FB00212846FFF725FB874E002130463F
:10127000FFF720FB854F0021384600F0C9F9012017
:101280004FF47041401C8842FCD32846FFF738FCDD
:10129000B1463046FFF734FC384600F0C5F94FF44C
:1012A0006020CDE912048DF8454001204FF004087C
:1012B0008DF8440010948DF8508010A92846FFF74F
:1012C000B1FC01231A4605212846FFF7FCFC012347
:1012D000022206212846FFF7F6FC012303220721FC
:1012E0002846FFF7F0FC012304220F212846FFF7D0
:1012F000EAFC384600F098F9684600F040FA614888
:10130000634E4C300090CDF80C80CDE90164802014
:10131000CDE904404000069080000790202008900E
:101320004FF44050CDE909046946384600F00AFA06
:1013300001212846FFF7C8FA0121384600F068F974
:1013400001212846FFF7B6FA47F230511594159857
:10135000401C15908842FAD301212846FFF7F2FC81
:10136000ADF82C40A04640F2DC5A4FF4007420E067
:101370005046CDF854801599491C15918142FAD3F5
:1013800030880D9908440D9070880E9908440E908D
:10139000B0880F9908440F90F0880C9908440C907D
:1013A00001212846FFF7CEFCBDF82C00401CADF80B
:1013B0002C00BDF82C00A042DAD30D98354A40F33A
:1013C000CF1633480A3006830E9941F3CF14448375
:1013D0000F9941F3CF1383830C9941F3CF1CA0F8ED
:1013E00004C0ACF5C05C40F2C371ACF59B7C8C458D
:1013F0000ED2A6F5C856363E8E4209D2A4F5C85480
:10140000363C8C4204D2A3F5C853363B8B4203D3FF
:10141000D18841F48041D180D188490407D41E4944
:10142000028B21F85C2F428B4A80808B88800021C0
:101430002846FFF749FA0021384600F0E9F8002174
:101440002846FFF737FA00214C464846FFF732FAA4
:101450000220C102401C8842FCD32846FFF750FB03
:101460002046FFF74DFB384600F0DEF8FFF736FA6E
:101470000A493C20087062B616B0BDE8F08700004B
:1014800000100240002401400028014008000240F2
:1014900012050020100A0020680C0020EC06002035
:1014A000F0B53F4B404C93F856503E4B042D5B6CCF
:1014B0001DD0256840F22D465D1B656043F6FB2577
:1014C000B3F5FA5F33DDB3F5FA4F30DC41F6AD1713
:1014D000A3F5FA535F4306EBA7364FF4B5777B438A
:1014E00005EBA31375105B10C4E9065321E043F626
:1014F000D017102641F26205BB4218DB44F2506758
:10150000BB420EDAA3F5645345F24C67D03B5F4310
:1015100006EBA736A66140F62476734305EB23233A
:1015200003E042F24713A361204BE36101E0C4E909
:10153000066540F2AE43936044F24C23401A1361B7
:1015400010605168884202DA4942884200DC11602A
:10155000106844F24C214843117D0841516A01440E
:101560005162106A814200DD5062516AD069814245
:1015700001DB084600E050622062116840F2AE4391
:101580005943137B194118410144B2F918008842AC
:1015900004DBB2F91600884200DC08B2F0BD00009E
:1015A000600000203C0100201401002085EB0100B8
:1015B00010B54FF40054204600F0ACF8002813D0CA
:1015C0000A49087840F008000870204600F014F836
:1015D0000021074800F01CF80648C17E012903D10C
:1015E0000021C1760121017710BD000066060020B0
:1015F000440002400C0B0020C10002D502490860E3
:1016000070470249486070470404024000000240ED
:101610000029016802D041F0010102E04FF6FE729C
:10162000114001607047000001684FF6FE721140E2
:1016300001600021016041608160C1603149314A2F
:101640000839904203D1486840F00F0006E02D4A67
:101650001432904204D1486840F0F000486070476E
:10166000284A2832904203D1486840F47060F5E778
:10167000244A3C32904203D1486840F47040EDE780
:10168000204A5032904203D1486840F47020E5E788
:101690001C4A6432904203D1486840F47000DDE790
:1016A000184A7832904203D1486840F07060D5E71C
:1016B000154A111F904203D1086840F00F0006E060
:1016C000114A1432904204D1086840F0F0000860DA
:1016D00070470D4A2832904203D1086840F4706088
:1016E000F5E7094A3C32904203D1086840F4704063
:1016F000EDE7054A50329042EAD1086840F4702084
:10170000E5E700000800024008040240406880B29B
:101710007047000001460020CA0001D5034A00E0DE
:10172000034A12680A4200D00120704700040240B8
:1017300000000240002A026801D00A4300E08A4308
:101740000260704730B5036847F6F07293430C6A45
:101750008A682243D1E904452C4322438C69224301
:10176000CC6922434C6A22438C6A22431A430260AA
:10177000CA6842600A6882604968C16030BD002161
:10178000016041608160C160016141618161C1614D
:10179000016241628162704710B5114C8CB000212A
:1017A0002046FFF735FF2046FFF73EFF0D4800902B
:1017B0000D480021CDE901016420CDE9030180201D
:1017C000CDE905010791089109910A9169462046E2
:1017D000FFF7B8FF01212046FFF71AFF0CB010BD3C
:1017E00058000240043801408407002010B5012150
:1017F0008CB0084602F064FB1E4C00212046FFF727
:1018000007FF2046FFF710FF1B4800901B48019080
:1018100000211020CDE902018020CDE904100691BD
:101820000791089109910A9169462046FFF78AFFBE
:10183000012202212046FFF77DFF01218DF82F10A4
:1018400004208DF82D008DF82E100E208DF82C0020
:101850000BA802F021F80F208DF82C000BA802F045
:101860001BF801212046FFF7D3FEFFF795FF0CB0D0
:1018700010BD000044000240043801402007002051
:1018800030B540F6AA21204AC184838B1488E31A1C
:101890009BB20F2B10D312888283037E002253B198
:1018A0001A4BB3F90A30062B05DB194B1B78022BB8
:1018B00003D0002B00D1828430BD164B40F68B251F
:1018C0005B6CA3F22D14AC420FD2428B521C92B22D
:1018D0004283642AF0D364224283B0F924208A42EE
:1018E00001DA02EB2111818430BD41F29414A3424C
:1018F000FADBB0F92430002B02DDA3EB211100E06C
:1019000000218184428330BDF80600206000002061
:10191000EF0600203C01002010B50446B0F902009B
:1019200043F6991148438113E06840F266625043E0
:1019300001EBA030E060B4F9001043F69912514376
:101940008A13216940F26663594302EBA131216198
:1019500004F0DEFC6061A18840F6AB220844401030
:10196000A0F515415539E062914205D9A0F5F8512D
:10197000FF39521C91421DD249F25451884202DD76
:10198000A0F5204002E0A0F5F850FF38206300EBFE
:10199000400040F34F002085B4F924104A429042A1
:1019A00001DA104602E0884200DD0846E083228426
:1019B00061848AE0A0F5FE42FF3A41F255518A4225
:1019C00014D8A2F6AA20206300EB400040F34F0099
:1019D0002085B4F924205142E183884201DA084687
:1019E00002E0904200DD1046404250E0A0F5D442B3
:1019F000AA3A8A4215D2A2F6AA20206300EB400040
:101A000040F34F012185B4F924004242E28320844F
:101A1000914201DA104602E0814200DC084660840F
:101A200053E0A0F5AA42543A41F256539A4215D2D5
:101A3000A2F6AB20206300EB400040F34F0020856E
:101A4000B4F924104A42904201DA104602E088427A
:101A500000DD08464042E083218419E0A0F5804281
:101A600041F254539A4215D2A2F6AA20206300EB09
:101A7000400040F34F012185B4F92400E083424245
:101A8000914201DA104602E0814200DC08462084DF
:101A900062841AE0A0F52852AB3A8A4215D2A2F627
:101AA000AA20206300EB400040F34F012185B4F9E8
:101AB0002400E08342422284914201DA104602E08F
:101AC000814200DC08464042A9E7B4F91E006FF4E9
:101AD000BF7148438013E080B4F92000484380136D
:101AE0002081B4F9220048438013608110BD704703
:101AF0001548164A4FF480410078042821D002F19D
:101B00003C03D08A9B88C01A00B22F2801DD001147
:101B100008E0002801DD002007E00D4B984201DAC3
:101B2000184602E0402800DD40209389184400B2A6
:101B3000884203DC40F26661884200DA0846908100
:101B40007047918170470000EF060020B404002028
:101B5000C0FEFFFF38B54B484B4902880B889A1AE4
:101B600092B20F2A71D30988484C01804FF0FF01CF
:101B7000E2884FF47A7355044FF4967002D516221A
:101B8000009103E0950403D515220091014670E011
:101B9000D50402D514220091F8E7150502D51322C9
:101BA0000091F3E7550502D512220091EEE7950565
:101BB00002D511220091E9E7D50502D51022009146
:101BC000E4E7150602D50F220091DFE7550602D59E
:101BD0000E220091DAE7950602D50D220091D5E795
:101BE000D50602D50C220091D0E7150702D50B22AD
:101BF0000091CBE7550702D50A220091C6E7950769
:101C000002D509220091C1E7D20702D00822009133
:101C1000BCE72289550702D507220091B6E7950750
:101C200002D506220091B1E7D20702D00522009129
:101C3000ACE7A27AD20702D004220091A6E7A289DB
:101C4000D40603D503220091A0E719E0140702D5BA
:101C5000022200919AE7540703D4940701D4D207D3
:101C600002D00122009191E700200346024601467E
:101C7000009002F031FEBDE838400248FFF71AB983
:101C800038BD0000040A0020F8060020100A0020D9
:101C9000F0B55948594982880B889A1A92B29C2A01
:101CA00064D30988818056490A880146002A0B7846
:101CB00043F0020156D11646524A1C0715680246E7
:101CC000127822F0020274D54F4C0746E4887F78E0
:101CD0005FEA845C02D547F0010701E027F00107C5
:101CE0004770A704477802D547F0020701E027F0C4
:101CF00002074770670401D4E70703D0477847F02D
:101D000008074770640603D5447844F0040404E0EF
:101D10001C0603D4447824F004044470EC0450D42A
:101D2000354C9A07247824F0100423D4324D42789D
:101D30002F7A2D78012A45F0100514D0022A16D0EA
:101D40002D4C042AA47804F1010C0CF0FF0C13D0E4
:101D5000072A25D0032A23D0052A21D0062A1FD0FE
:101D600021F0100142E0B90702E00570F0BD39072B
:101D70000029FADB0470F0BDFA0601D41A060AD570
:101D80000170022C04D280F802C0BCF1020FF2D321
:101D900041F080012AE021F0100101708670F0BD51
:101DA000877A7F06F7D5032C04D8017080F802C02B
:101DB000F0BD0FE05107D8D51906D6D443F0800105
:101DC00014E002704178CB0701D18907F0D522F0E9
:101DD00010010BE0E9040BD49907E9D4818AC829E2
:101DE00002D2491C8182E3E743F00A010170DFE778
:101DF00002708682DCE70000D0060020F806002092
:101E0000FA06002098020020100A0020094944F632
:101E100048000880091D46F648000880091D41F663
:101E2000CC4008800348001F018841F02001018058
:101E300070470000182C0140084946F668000880E9
:101E4000091D0880091D41F2555008800348001FF4
:101E5000018841F02001018070470000182C0140EA
:101E600010B5C28800210AB1032206E002890AB136
:101E7000022202E0428912B10122027000E00170E8
:101E800004784FF4804344F6206244B1012C06D01C
:101E9000022C07D0032C01D14180818010BD4380EA
:101EA000828010BD41F23331418040F6B731F4E712
:101EB00030B5B1F86A5000231A240D22854202DCA5
:101EC000B1F9680030BD4D88854202DBB1F90000F0
:101ED00030BD01EB82056D88854201DD144601E0CD
:101EE00013DA134604EB03024FEA52029A42F0D18E
:101EF00001EB830231F8231054889288521A001B98
:101F0000424301EB622000B230BD31F9220030BD06
:101F1000054920B1086940F0800008617047034816
:101F2000486003484860704700200240230167452D
:101F3000AB89EFCD06494FF47A70CA68D20705D055
:101F4000401E0004000CF8D1FF20704700207047AD
:101F50000020024011480321A0F14C0280F8361005
:101F6000002151810E4A1186D162D183118451849E
:101F700081620C498A6CB2F5206F01DBA322826278
:101F8000897A11B1816A49428162C16A41F3910142
:101F900081628803044948627047000060000020A5
:101FA0001C0500203C01002064080020044900209A
:101FB00048810881C862886202494862704700000F
:101FC000600000208C080020F0B53B4988894A89D0
:101FD000801A80B20F2866D388894881CA89374819
:101FE0000B3A272A26D28A7822BB8268364B42F4E3
:101FF00080728260324A354C354D12785607314A2C
:102000000AD4344E36881680334A12881A80334AEE
:1020100012882280324A09E0324E36881680324ACF
:1020200012881A80314A12882280314A12882A8006
:1020300001228A702F4B304D19469A7F0968802AF9
:1020400032D302F01F0255F8222011422CD08268B0
:1020500022F48012184E8260123614461215B77898
:10206000521C62F38617254AB77093F816C017788A
:10207000BCF1800F27F0020608D30CF01F0C55F8B6
:102080002CC011EA0C0F01D147F0020616701A7E1F
:10209000802A0DD302F01F0255F82220114207D1E9
:1020A00044F400218160F0BD826842F48012D1E7DF
:1020B00024F40021F6E70000EC060020980200203E
:1020C0003C010020AC040020AE040020B00400203D
:1020D000B20400209C0400209E040020A0040020E4
:1020E000A2040020A4040020A6040020A8040020CC
:1020F000AA040020CC050020F88F0008B4040020BA
:1021000070B5204881890289891A89B20F292FD395
:10211000818901811C4B1D4819465D7A06681C4C5B
:10212000096846F00402802D07D305F01F0554F816
:102130002550294201D126F0040202609A7B802AB0
:1021400017D302F01F0254F82220114211D1026865
:1021500022F002020260DA7A802A0ED302F01F0215
:1021600054F82220114208D1016821F008010160D1
:1021700070BD026842F00202ECE7016841F008011C
:10218000F5E70000EC060020CC05002098020020B6
:10219000F88F0008F0B51D4C1B4A4FF0010C94F865
:1021A0003B5094F80AE0144692F83C3094F83840DA
:1021B0002B43651CEEB2154D95F83D700025BEF120
:1021C000FF0F0AD0BEF1000F06D18B4213D155701C
:1021D0000C2C01D282F83860F0BD834202D182F823
:1021E00001C0F5E78B42F7D15570B80709E000BF91
:1021F00082F83850F0BD8342FCD1F84382F801C028
:1022000080070028F4D0F0BD3C0400203C010020F1
:10221000F0B5CA78002502F00F03D20601D58A78FE
:1022200013430A784FF00F0E12F0FF0F4FF0010228
:102230001CD004680F8802FA05F63740B74211D166
:102240004FEA850C0EFA0CF724EA070703FA0CF4A0
:102250003C43CF78282F02D0482F02D002E04661BD
:1022600000E006616D1C082DE4D304600C88FF2C8F
:102270001ED944685FF0000606F1080702FA07F568
:102280000F882F40AF420FD14FEA860C0EFA0CF7A1
:10229000BC4303FA0CF73C43CF78282F00D14561AB
:1022A000CF78482F00D10561761C082EE4D3446016
:1022B000F0BD0000F0B5144C002801DAE36900E03D
:1022C0006368420D120185B2C0F301579540C0F317
:1022D0000346032F05D0C2020AD50322B24093431E
:1022E00007E023F07062636823F07063636002E0CC
:1022F000AB4343F0706201B12A43002801DAE26186
:10230000F0BD6260F0BD0000000001400246002008
:1023100092680A4200D00120704741617047016114
:1023200070470AB101617047416170470F4A104B15
:1023300092F838105B5C834201D1012004E00D4B20
:102340005B5C834203D1002082F83A0070470A4B5D
:102350005B5C834201D18120F6E7084B595C8142E6
:1023600001D18020F0E70320EEE700003C010020CF
:10237000B8930008CA930008BE930008D0930008E1
:102380000A4810B501784FF000024C0708494FF099
:10239000FF0389684FEA017105D5002901DA8272CD
:1023A00010BD837210BD0029FBDBF8E73C01002063
:1023B00098020020F0B5194E194C0022E31CA6F13A
:1023C000060CB75CA518ED78FF5C0D430F43BD42CA
:1023D0001FD01CF80270FF5C0F43BD4219D0154698
:1023E0000023A618F6780E43C6545B1C1CF8022086
:1023F000DBB2062BF5D3C17881700179C170002161
:102400004218491C15711CF80550C9B20629F7D3AA
:10241000F0BD521CD2B2032AD3D3F0BD8A8B000880
:102420003C04002010B502460021064B06205C1833
:102430006478944200D10846491CC9B20629F6D3F3
:1024400010BD00003C010020214810B590F8671035
:1024500000222048012936D11F49898899BB1F498C
:102460001E4B4C6C40F6B831B3F86E308C4227DD11
:102470001B49097821BB90F82711491CC9B280F883
:102480002711C8291CD380F827210146D0F82C41F8
:1024900091F82811A34203DD052908D2491C01E067
:1024A00041B1491E80F82811C9B2052902D3012182
:1024B00080F82611191B074C2C3C6162C0F82C31A6
:1024C000B3F5FA6F03D280F8262180F8282110BDD9
:1024D000680C002098020020C60500203C01002066
:1024E000EF0600204FF4C0428260002141620E22BC
:1024F000828141F262020261082282824FF46042CC
:10250000C28201834FF07842C0E9072140F6C4112E
:1025100001807047B0F90010B0F90220891A4160BB
:102520000269037D4A431A41436A13444362026AC3
:10253000934200DD4262436AC269934200DA42621A
:102540008268436A4A43017B0A410B41D118B0F9C2
:1025500018208A4201DA10467047B0F91600884206
:10256000FADC08B27047000010B514481449B0F8FE
:102570008C200B889A1A92B2B2F5437F1DD9098834
:10258000A0F88C10B0F88A1020F8581F002242865C
:102590000C480D4CC2888280C180C3898381248904
:1025A000891AA4B2C4818160E11A0161074A818A53
:1025B000C182928A8282511A816110BD3C01002041
:1025C000F8060020300C00201C05002060000020D0
:1025D00009480A49B0F8AA200B889A1A92B241F623
:1025E00084639A4206D3098820F8AA1F4188818013
:1025F00000214180704700003C010020F8060020C7
:102600000D480178C90702D00C49098801E04FF64E
:10261000FA71C1650949012010390880074824383A
:10262000018841F00101018004481838018821F037
:1026300018010180704700003C0100202404004084
:102640000A49D1F8902012B1521EC1F8902031F8F9
:102650008A2F521C21F81A294A6A521C4A628A8F10
:10266000521C8A8701F8380C704700003C0100209A
:102670001CB52D4890F83B3090F83C20934252D046
:1026800000248DF8044053408DF800309DF8003050
:102690000122012B08D09DF80030022B09D09DF8B3
:1026A0000030042B0AD00DE01F498DF8042044317E
:1026B00008E01D498DF80420463103E01A498DF8E1
:1026C000042048319DF80420012A2CD190F83D3097
:1026D0009DF80040154AA34217D090F83E309DF86F
:1026E0000040234208D0B0F84C30A0F84A300B88A4
:1026F0001488E31AA0F84C3090F838302BB1B0F8B9
:1027000040301488E31AA0F8423012880A80A0F8FA
:10271000402010F83E1F9DF80020114300F80119D9
:102720009DF8001001701CBD3C040020F80600203C
:1027300070B5344D40212846FFF7E8FD8400802124
:102740002846FFF7E3FD44EA4004A9152846FFF7B1
:10275000DDFD0443E1B22C4C94F870508D4250D012
:102760004D4084F87010012D03D0022D01D0042DAE
:1027700047D194F87400A84384F8740094F8732047
:10278000AA420FD084F8735094F8722001238B4032
:102790001A4207D11A4384F8722094F87110491C28
:1027A00084F8711094F87110042928D330B10128ED
:1027B00011D002280FD004280DD012E01348C18890
:1027C00021F04001C1802078002184F83B1020F0E6
:1027D0006000207005E0217841F02001217084F82C
:1027E0003B000B4994F83B0091F82720904204D01D
:1027F00081F8270007492020087000F00DF884F8C0
:102800004C5070BD001001403C010020100A002017
:10281000680C0020EC06002070B50D4D40212846C4
:10282000FFF774FD840080212846FFF76FFD44EA1E
:102830004004A9152846FFF769FD04430548072110
:1028400000F8704F0171002141708170C17070BD3E
:10285000001001403C01002070B5344890F83A1057
:10286000CA43920761D001F0030280F8392090F842
:102870003D305B061B0E80F83D30012A01D0812AD5
:1028800002D15B1C80F83D300278D2074DD0DBB21C
:1028900003F00102C3F34004A24246D1B0F84E4017
:1028A0000025641CA0F84E40204CA0F8505090F831
:1028B0003E60A47AB24202D080F83E200DE0A60726
:1028C000B6EB837F02D080F83F5006E090F83F30AF
:1028D000642B02D25B1C80F83F3090F84030642BB0
:1028E0000CD25B1CDBB280F84030022B06D204F025
:1028F0000103934202D1022280F84020012901D035
:10290000002912D190F83820C16D00EB820291614C
:102910000163D0E906121144D0E908231A44114496
:10292000826A1144C26A1144416370BD3C010020B7
:10293000FEE700002DE9F04F00BF00209E4E9F4AA9
:10294000A6F51271A6F5BE79A6F1440B06F1440E68
:10295000804601F5E074A1F1780301F5457A1D5C2C
:1029600015F0C00706D0402F51D0C02F77D0802F50
:1029700076D004E115F01F0504D0154440F080071F
:102980002F7201E082F80880012826D0022824D086
:10299000032822D0042820D008281ED010281CD0BC
:1029A000874D55F820C0DCF8005054F820703D40A9
:1029B000CCF80050824D55F820C0DCF8005056F895
:1029C00020703D43CCF800501D5CAD0659F82050F6
:1029D0002F6813D53AF810C03EE051F820502F6808
:1029E00054F820C007EA0C072F6051F820502F68D8
:1029F00056F820C047EA0C072F60E5E7DFF8B8C1BA
:102A00000CF1F00C5CF820C007EA0C077EE015F032
:102A10001F0504D0154440F080072F7201E082F8B2
:102A2000088001281DD002281BD0032819D00428B3
:102A300017D0082815D0102813D0614D55F8205014
:102A40002F6854F820C007EA0C072F605C4D55F83A
:102A500020502F685BF820C047EA0C0756E00BE0D7
:102A600056E051F820502F6854F820C007EA0C07B0
:102A70002F6051F82050ECE715F01F0505D01544E4
:102A800040F0800785F8217001E082F8218001285C
:102A900025D0022823D0032821D004281FD00828BD
:102AA0001DD010281BD0464D55F820C0DCF8005032
:102AB00054F820703D40CCF80050414D55F820C0EE
:102AC000DCF800505EF820703D43CCF800501D5CEF
:102AD000AD0615D53A4D3AF81070CC3514E051F8E2
:102AE00020502F6854F820C007EA0C072F6051F8D7
:102AF00020502F685EF820C047EA0C072F60E6E7F9
:102B00002D4D3AF81070E03D55F820502F6036E01A
:102B100015F01F0505D0154440F0800785F8217099
:102B200001E082F82180012830D002282ED003282D
:102B30002CD004282AD0082828D0102826D0204DB0
:102B400055F820C0DCF8005054F820703D40CCF817
:102B500000501B4D55F820C0DCF80050164F883748
:102B600057F820703D43CCF800501D5CAD06B1D441
:102B7000114F3AF81050E03F57F820703D60401C6C
:102B8000C0B21128FFF4EBAEBDE8F08F51F8205031
:102B90002F6854F820C007EA0C072F6051F8205026
:102BA0002F68DFF814C00CF1880C5CF820C047EAED
:102BB0000C072F60D9E7000084920008CC050020A4
:102BC000809000084FF40771C1824FF4586101836F
:102BD00040F6145181837047F0B5C48AB0F90060A3
:102BE0008681B0F90250C581B0F904300227002176
:102BF00001220382AB4204DBB54202DDC780428181
:102C00000CE0B34204DBAE4202DDC78041811CE030
:102C10009D4205DBB34203DDC2804781018115E09F
:102C2000B54204DB9E4202DDC280418105E0AE4236
:102C300005DB9D4203DDC1804281078106E09E42A3
:102C400004DBAB4202DDC18047810281C388458934
:102C500000EB430700EB4505BB89AE899B1B0FFAD0
:102C600083FEA0F812E00689AB8900EB460CBCF8A5
:102C70000CC0A3EB0C038382B0F91830B7F90CC079
:102C8000A3EB0C0CB4EB4C0F04DA80F82010A3F18A
:102C9000A10113E0A64503DD80F82010B9890BE0FF
:102CA00026B1012E04D0022E10D004E0062100E04F
:102CB000052180F82010A989091B6D31418309B2D3
:102CC000B1F5586F04DB5B1E438304E00421F0E799
:102CD000002900DC4283418B8183F0BD0B49002237
:102CE00088760A62CA614A62094A32F9103002EBF8
:102CF00040028B62B2F90220CA62064A32F8100022
:102D00000882A1F86000A1F862007047EC01002081
:102D1000E2930008D69300082DE9F05FF748F849E0
:102D200082880B889A1A92B20F2A44D3098881802C
:102D3000F449824601270888F34CF44E002578B305
:102D4000401E0880E573F249A5622068B1F90210BF
:102D5000430742F6AA2218D4F38843F40053F380C1
:102D6000EB4B1B789B0709D5A36823F08003A36076
:102D7000A4F87C5084F87E5084F87F50C30404D4B7
:102D800084F8F070C4F8EC5003E084F8F050430786
:102D900007D4914205DB84F8F470A4F8F25004E003
:102DA00010E084F8F450430703D4914201DBC007DC
:102DB00003D084F81151BDE8F09F84F81171A4F894
:102DC0001251F8E7B4F8180143F69821884202D26C
:102DD000401CA4F8180101F095FDDFF8388398F83D
:102DE000500010B1FEF770F905E0C44818380178BA
:102DF00021F001010170FFF727FB00F0C7F9C64879
:102E000041F26801D0F844C04FF400608C4501DB0A
:102E1000C24904E0BCF57A6F02DAC049091D0860B6
:102E200098F85100DFF8E0B2C107BD48DFF8F4922E
:102E30004346ABF12C0B38D0817B802931D32178EC
:102E400089072ED4E27B8BF80520B14A594692F8C7
:102E5000008028F0020882F80080A84A183A5580BD
:102E6000556192F8008028F0010882F80080B2795C
:102E7000520611D44A89B2F5FA7F03D2521CABF83C
:102E80000A2012E040F63C70844501DD002001E19B
:102E900008208BF80370FDE0CD700020ABF80A50DD
:102EA000F8E08BF80350ABF80A50A1680A0501D589
:102EB0000820EFE093F83FE09C465FEACE7240D0F6
:102EC000E27B8BF80520437A802B44D323785B0781
:102ED00030D4F3889B0403D521F02000A06030E0BB
:102EE000864B41F02001183B5D805D6193F800C086
:102EF0002CF0010C83F800C0A160C17D802909D3AA
:102F000001F07F0300684FF00041D940084201D131
:102F1000277100E025712079C00702D15FEA8E7029
:102F200005D50320032A01D08BF80870B2E00020F9
:102F3000A562AFE021F02000A060F08820F40050EE
:102F4000F08094F8260101280AD09CF8630048B16B
:102F5000FDF77AFF0FE0206840F004002060BBE737
:102F6000092097E0A068C10502D520F0080001E023
:102F700040F00800A06094F8462043F233304FF44C
:102F800080477AB143F69911012A1DD0032A99F896
:102F900000206548C2F3810223D0012A39D0022AD9
:102FA00037D033E099F80010C1F38101012908D02E
:102FB000022906D043F26661A4F81411A4F8440073
:102FC0002BE0A4F81401F9E799F80020C2F381027C
:102FD000012A03D0022A01D043F21E50A4F81401A2
:102FE00019E0012A0BD0022A09D090F856000428D3
:102FF0000CD0A4F8147100BFA4F844700DE0A4F83C
:10300000147190F85600042805D0F5E7A4F814715F
:1030100001E0A4F81471A4F84410FEF755F83748FD
:1030200018380178C90701D0418801E03848818803
:10303000AAF8121008B2B4F944104843C0F38F3113
:103040005846ABF81210B94200D94782374909787F
:10305000C90605D5428A41F233318A4200D2418203
:103060002189C1F3C002C1F300218A4205D1428AFD
:1030700040F6CC418A4200D94182B17AC90700D0DA
:103080004582BBF81200A06200287FF7FFAE2848F7
:10309000057002209AF81A1099B9022824D080B13C
:1030A0001D4A11788D0608D5B5796D0605D51F4DD9
:1030B0002D78ED0965F386111170F18821F40A610C
:1030C000F1801549496C4E290ADBF1880A0607D5BB
:1030D00021F08001F1800E490A7822F002020A7084
:1030E0008AF81A00E07366E6B9F83820002AD7D1CA
:1030F00043F69822A9F83820D2E7000020090020E2
:10310000F8060020FA06002098020020100A00208D
:10311000C6050020680C00203C010020100C014076
:10312000CC050020B404002060000020D006002060
:103130000C07002070B500230C8863F30F020125F3
:1031400005FA03F6344206D0C3F10F0605FA06F17C
:10315000114361F30F025B1C102BF1DB028070BD89
:1031600070B500230C7863F30702012505FA03F616
:10317000344206D0C3F1070605FA06F1114361F3A4
:1031800007025B1C082BF1DB027070BDF0B51F4815
:1031900090F866301E48012B816821F4006232D11C
:1031A0001C4BDE8874062ED41B4D0F054FF0000417
:1031B000B5F902501ED4194A526C642A11DC40F64B
:1031C000386295420DDAB2040BD4027852070ED45D
:1031D000B0F8D42040F6B835AA4203D2521CA0F869
:1031E000D420F0BD41F4006181605C81F0BDA0F8A5
:1031F000D440F0BD41F2CD018D42FADD997AC90784
:10320000F7D18260F3E78260F0BD0000680C002017
:1032100098020020100A0020C60500203C01002072
:10322000F0B5364D364F044695F83B0097F83B1005
:1032300023780843EE1C6278834205D1E07811467A
:10324000FEF7A8FF207908E094F802C084450CD16D
:10325000E1781046FEF79EFFE07905F82F0F2878F9
:10326000805D6870287BE877F0BD82421DD16146A1
:103270001846FEF78FFF95F84E1095F83B008142F7
:1032800007D1B97A09B1A17900E0617985F82F10E9
:103290001EE06978012901D0A17922E0617927E057
:1032A000297841F00401297012E0E1788142DBD1F4
:1032B00019466046FEF76EFF95F84E1095F83B00F4
:1032C00081420AD1B97A09B1617ADFE7217ADDE773
:1032D00015F82F1F895D6970C5E76978012906D047
:1032E000617A85F82F10B97A0029F1D1D8E7217ACF
:1032F00085F82F10B97A0029EAD0D1E73C040020E4
:103300003C0100200B48017821F0020100F8381B35
:10331000002100F818194177817733218185418593
:1033200008214184012100F81F1C034880F839104E
:10333000704700003C0400203C0100200D4900B50E
:103340000B4851F8012F40F8032F898881800848E5
:1033500001210930FFF72EF8054802211330FFF74D
:1033600029F8034804211D305DF804EBFFF722B86B
:103370003C0400203C010020094944F64800088034
:10338000091D46F648000880091D41F21110088009
:103390000348001F018841F02001018070470000B0
:1033A000182C01402DE9F047664C674B0025A078AA
:1033B0000126654A103305287ED2DFE800F00313AA
:1033C000113E1100108820F0010010801D805F4820
:1033D0000580001F0580001F0580FFF7CDFFA67048
:1033E000BDE8F087594941F244401C3908805749EB
:1033F00045F6580024390880091D47F25800088016
:1034000052492020283908800020401CC0B273286F
:10341000FBD3FFF7B1FF4C4984F85C502C3147F6E1
:10342000906008804848143006801D80108840F065
:10343000010010800220A070D2E700215FF001009F
:1034400004EB410204EB4003B2F85020B3F85030D3
:103450009A4200D20146401CC0B20628F0D33C4834
:10346000405C84F83900FFF74DFF1D2000F0F3F9B0
:1034700000F076F8374E38484FF4807996F83B10D4
:10348000012904D002291BD0042930D047E0402173
:103490008046FEF73BFF870080214046FEF736FF5F
:1034A00047EA400749464046FEF730FF074347F0EA
:1034B000010084F83B0000E03DE0224809302CE0A8
:1034C00040218046FEF722FF870080214046FEF71C
:1034D0001DFF47EA400749464046FEF717FF0743EE
:1034E00047F0020084F83B001648133015E04021F5
:1034F0008046FEF70BFF870080214046FEF706FF5F
:1035000047EA400749464046FEF700FF074347F0B9
:10351000040084F83B000B481D3002F0D3FD94F802
:103520002F0086F838001D2000F0ABF90420A070B1
:103530000A48057054E7108820F0010010801D80B3
:10354000A5704DE73C040020000800403C2C0140E1
:10355000908B00083C01002000100140EF06002085
:103560002DE9F041344C14F82F0F344DE072402116
:103570002846FEF7CBFE860080212846FEF7C6FED1
:1035800046EA4006AF1539462846FEF7BFFE064319
:10359000207BF1B22F3C814215D084F83C004021C1
:1035A0002846FEF7B3FE860080212846FEF7AEFED1
:1035B00046EA400639462846FEF7A8FE064384F848
:1035C0003B60FFF755F81E4D95F83B00012827D0CA
:1035D000022828D0042829D0174894F83B10273017
:1035E000085C04F8300F14F80109FEF71BFF04F81B
:1035F0002F09A87A00B10120607001F00FFA94F849
:103600004E0094F83B10884206D094F83800062803
:1036100002D2401C84F8380084F84E10BDE8F081D6
:103620000548093004E00448133001E002481D3029
:10363000BDE8F041FFF7F4BD3C040020001001405C
:103640003C0100202DE9F041524991F87200AA286E
:103650007ED191F8730055287AD14F4C00200A5C36
:103660002254401CC0B27428F9D34C4E2069C6F8CD
:103670000100A08AA6F80500D4F81600F060D4F87E
:103680001A003061D4F81E001234706102F0C0FCE0
:103690004349608A888102F0D5FC207D123CC00736
:1036A000307802D040F0040001E020F004003D49F1
:1036B00030704FF480403C4D886114F8280F85F835
:1036C0002000608B6880A08BA880E08BE880208C35
:1036D0002881608C354F688194F8240087F8D200E7
:1036E00014F8011C304686F83B100026C0F89460A0
:1036F000FFF724FE2E48A18E0183E18E4183218FA6
:10370000818394F84210283C012908D0022901D075
:10371000032909D0297821F00C01083107E0297824
:1037200021F00C01091D02E0297841F00C012970FB
:1037300094F86E20012162B1012A01D0022A0BD037
:1037400087F8461094F864301A4A4BB1518108E06A
:1037500014E087F84660F5E7022287F84620F1E793
:10376000568194F8701001290AD094F86D1051B167
:1037700001290BD04FF48051A0F87610BDE8F081FC
:1037800044F21C71F8E74FF40051F5E741F255514E
:10379000F2E7000000FC0008680C00203C0100205B
:1037A00060000020000C0020B404002098020020DB
:1037B0001C050020100A00207CB50121082000F023
:1037C000A3FB4FF48070ADF8040010248DF807407F
:1037D00001208DF8060001A91548FEF719FD012109
:1037E000092000F091FB01211248FEF763FD08203B
:1037F000ADF8000004208DF803000F4E03258DF86E
:10380000025069463046FEF703FD08213046FEF7B8
:1038100084FDADF800408DF803408DF802506946F4
:103820003046FEF7F5FC10213046FEF776FD7CBDF4
:103830000014014000023000000C0140FEE7704718
:1038400000F01F02012191404009800000F1E020BA
:10385000C0F88011704700F01F020121914040091B
:10386000800000F1E020C0F88011704700F01F02D6
:10387000012191404009800000F1E020C0F80011D2
:10388000704700F01F02012191404009800000F1C3
:10389000E020C0F80011704770B50F23C47801789C
:1038A0000122F4B1144C2468457804F4E064C4F5B2
:1038B000E064240AC4F10406E3408478B5401C4067
:1038C0002C4301F1E021230181F80034007800F05D
:1038D0001F018A404009800000F1E020C0F800216B
:1038E00070BD01F01F0082404809800000F1E02017
:1038F000C0F8802170BD00000CED00E002490843D3
:1039000002490860704700000000FA050CED00E075
:103910002DE9F05F00261D20FFF792FF6C4CDFF8C9
:10392000B4B1A4F1B000A77E90F83810DFF8A8E198
:10393000DFF8A8A100258F427ED0E776A176626AE3
:10394000036B5A434FEA12499BF80820120702D52D
:103950001EF8012000E00A4694F812C0BCF1010FE5
:1039600009D004EB4206B6F902C0C4F828C0B6F983
:103970000460E6620CE043F6FF7CC4E90A5C90F860
:103980003DC05FEACC7C01D012B102E0052A00D133
:10399000012600EB47074FF0804CBF893F04B7FB7F
:1039A000F3F3E361476BBCFBF7F7276294F813C0AE
:1039B000BCF1000F06D0BCF1010F05D03B4403EB76
:1039C000D3735B10636201E03B466762DFF810C1AE
:1039D0004FF6FF7707EA8307ACF808709AF8007093
:1039E00090F80A8090F83DC0082F08F003070CF00B
:1039F000030C05D067450BD1B8F1000F05D008E0E6
:103A0000674505D0B8F1000F03D05B42636200E068
:103A10006562C6B1636A002B03D006DD228D05E026
:103A20000AE0304B33F8122000E0A28DA4F86020A9
:103A3000227822F0200222709AF80020042A07D06F
:103A4000082A05D012E0B4F8603003EB0902EDE774
:103A500080F8405065629BF80800000701D51EF809
:103A60000110204830F81100A4F860001E49606A77
:103A700009883E314843B4F8601001EB204006B29B
:103A80001D20FFF7F3FE606A002807D021784FEA77
:103A900081600ADD002804DAA08D09E0B4F8600036
:103AA00006E0E06AB04208DB0CE0002802DA208D74
:103AB000208208E0A06AB04204DD208241F02000AC
:103AC000207000E02682257565752586BDE8F09F8B
:103AD000EC01002098020020C4930008EF060020AB
:103AE000E8090020D69300082404004043184FF44E
:103AF0008042934210DD904202DD104600210BE02F
:103B0000914202DD0020114606E08003B0FBF3F095
:103B100000B2C0F5804109B241EA00407047F0B5FB
:103B2000002240F2AE440E2584604262858144F258
:103B30004C2608270661878243F6FF7CC282A0F8E4
:103B400018C040F249234FEA8C3E4360C0E9072E7B
:103B50008C604A628D810E618F82CA82A1F818C082
:103B60004B60C1E9072EF0BD002141620949816027
:103B70000E2181814FF6BF510161082181824FF4EE
:103B80004041C18243F6FF7101830907C1610249C7
:103B900001627047638A010000C0FF0F064941F6C9
:103BA000A260088005480168054A01F4E0611143FC
:103BB0000160BFF34F8FFEE7442C01400CED00E0A5
:103BC0000400FA0538B501210D2000F09DF94FF4ED
:103BD000E060ADF8000018248DF8034003258DF84F
:103BE000025069460D48FEF713FB4FF46040ADF8F4
:103BF00000008DF803400A4C8DF8025069462046BB
:103C0000FEF706FBA014ADF8000048208DF8030075
:103C100069462046FEF7FCFA38BD00000008014066
:103C2000000C0140F0B50121CE028DB0304600F00D
:103C30006BF9594F384601F063FB08A801F08CFD81
:103C40004FF45860ADF824000024ADF82040202047
:103C5000ADF82200ADF8264008A9384601F02EFD47
:103C60000021384601F081FD4FF6FF71384601F022
:103C700086FD01220021384601F012FD012138465F
:103C800001F0FAFA04A801F012FBADF81060701010
:103C9000ADF81200ADF81440A220ADF81600700087
:103CA000ADF81800ADF81A40ADF81C4004A938462C
:103CB00001F0ECFA6025ADF80050ADF80440ADF825
:103CC0000840ADF80C40ADF80240ADF80640ADF844
:103CD0000A40ADF80E406946384601F0D1FB69460E
:103CE000384601F013FC6946384601F059FCADF83E
:103CF00000500125ADF8045040F61450ADF8060010
:103D0000ADF80840ADF80C40ADF80250ADF80A40EF
:103D1000ADF80E406946384601F086FC0121384670
:103D200001F0CEFA0821384601F0EAFB3146384668
:103D300001F02CFC0821384601F070FC3146384671
:103D400001F0A4FC7021384601F0ADFC18208DF87C
:103D50002C008DF82D408DF82E408DF82F500BA89B
:103D6000FFF79AFD0C480C30018841F0800101807A
:103D700009481430018841F001010180001F0480CE
:103D80000121384601F0A6FA8DF828500121384665
:103D900001F0AAFA0DB0F0BD002C01407047000000
:103DA00070B50189C1EB411101EB4101CA0B4281A0
:103DB0000B49104603F0E2FC09480C38B0F90C201E
:103DC0000168B0F90E4001FB02F54368614303FB53
:103DD000145503FB0211AD138913C0E9055170BDE1
:103DE000F409002040F213414160082181608621DE
:103DF000C1604FF48041016149424161002101628B
:103E0000C16270470162704710B501884288891A03
:103E100009B20183B1F5005F02DBA1F5804104E046
:103E200011F5005F02DC01F580410183B0F9182033
:103E300041685143C1618368846A5343C2681B125D
:103E4000624303EB2222036A1A44114402628A137A
:103E5000426241698A4203DB01698A4200DC114601
:103E60008A1AC0E90A21028E4FF40373594302EB08
:103E7000A13202860B4A1278082A04D10A4A136F2B
:103E800003EBA1311167B0F93010B1F5804F02DDBD
:103E9000A1F5804103E0002902DA01F580410186A5
:103EA00010BD0000EF060020240A0020034A5168DC
:103EB00021F440410143516070470000001002406E
:103EC000044A0029516901D0014300E08143516156
:103ED0007047000000100240044A0029D16901D057
:103EE000014300E08143D1617047000000100240AF
:103EF000044A0029116901D0014300E081431161A6
:103F00007047000000100240044A0029916901D066
:103F1000014300E0814391617047000000100240BE
:103F2000044A0029D16801D0014300E08143D160F7
:103F3000704700000010024030B524494A6812F072
:103F40000C03234A03D0042B01D0082B26D0026097
:103F50004A680F231F4C03EA1212A35C0268DA407E
:103F600042604B68072505EA1323E35C22FA03F35A
:103F700083604B6805EAD323E35CDA40C2604B6898
:103F8000032403F4404104EA933303EB9161114BA2
:103F90001B1F595CB2FBF1F1016130BD4A680E4B49
:103FA0001A404B68140103F4803303D5C2F38342F3
:103FB000113202E0022404EB924213B14B689B03DE
:103FC00001D5064B00E0024B5A43C0E70010024007
:103FD00000127A000400002000003C0800093D00A7
:103FE0002DE9F041274CA61540212046FEF78EF919
:103FF000850080212046FEF789F945EA40053146D3
:104000002046FEF783F90543EDB240212046FEF736
:104010007DF9870080212046FEF778F947EA4007BE
:1040200031462046FEF772F90743F8B2A842DBD1C9
:1040300040212046FEF76AF9870080212046FEF7DE
:1040400065F947EA400731462046FEF75FF9074326
:10405000F8B2A842C8D140212046FEF757F98700A0
:1040600080212046FEF752F947EA400731462046B4
:10407000FEF74CF90743F8B2A842B5D12846BDE88F
:10408000F08100000010014010B50268416802FB99
:1040900002F301FB01330D4CA34211D91B0E0E3B61
:1040A0000B4C9BB212B234F8133009B25A43594345
:1040B00042F38F3241F38F31C0E90221012102E046
:1040C000C0E902210021017410BD0000E10BBF0E08
:1040D0009C8700082DE9F05FF748F84902880B88B3
:1040E0009A1A92B20F2A7AD309880180F4480246BC
:1040F0008189D2884B0703D48B0701D4CB0702D028
:1041000042F4007201E022F40072C2808146080786
:1041100002D44846C90604D5B9F8061041F0010199
:1041200002E0C18821F00101A9F80610E448FDF77A
:1041300097FEE4484FF4804AB0F93A10514502DA4C
:10414000491C418702E0DF49A1F83AA0DE4E41F662
:10415000CC40DE4CB16C814203DDA06820F0100041
:10416000A060DB49DB4F0025088820B1401E088095
:10417000E5733D7027E0B9F8060042041BD4B9F896
:104180000C10CA0617D4090715D4010613D48106EA
:1041900011D401050FD4410603D5CF49097809068A
:1041A00009D5410707D4C10505D4010703D481040B
:1041B00001D4C00607D5C948E573C9493D70C58318
:1041C0000D8080F82A50E28FC648C74942B1521E7E
:1041D000E287027822F002020270E5730AE08AE0C8
:1041E000027842F0020202703878012803D1087880
:1041F000062800D13D703878DFF8D0B24FF00108C2
:10420000ABF12C0B0A2878D2DFE800F0F8750575C1
:10421000F7F67577DFF5E07B09281AD0DFF8CC9246
:10422000022875D0B4F8400010B399F8680040F641
:104230003A22012822D0C4F8D85084F8EA50CBF8AA
:104240002050B4F9301001F21D50904226D81023AE
:1042500025E099484430FEF745F9FDF77BFE716C87
:10426000CBF8281041F27C510920CBF81810A6E1B8
:104270009F4841892186A4F8408015E09D48C4F8F4
:10428000D80084F8EA80B4F9301001F21D5393424B
:1042900001D8102300E02023102202E02023102266
:1042A000002000F025FB208699F86810924A012929
:1042B000716C40F2DC504FF4927311D0814204DAF9
:1042C0008B48B0F90A00984211DBB4F8403040F650
:1042D000C4105B1C9BB2A4F84030834207D20EE0AE
:1042E000814208DA8248B0F90A00984203DA3D7048
:1042F00084F8EA505583BDE8F09FD2E008E07148A9
:10430000C0680028F7DC45F2F0508142EFDAF2E7AE
:10431000706CCBF828008BF80780784FA4F84050D9
:1043200084F8EA50797F5E4699B1F87FE0B3208D3A
:10433000B4F9301000B20A23052200F0D9FA208621
:10434000FD777D77B4F9300050453ADDA4F830A010
:10435000D1E700B26A4901F021FCA4F8E400A16AA7
:10436000814200DA084600B2B08299F84D10002967
:10437000B4F9301002D03623052202E040F2471390
:10438000102200F0B5FA2086B4F91601B4F9141120
:1043900088420ADA317901F10101C9B23171042987
:1043A000D0D33571401C02E007E003DD801EA4F885
:1043B0001601C7E7A4F81611C4E740F2666020862C
:1043C000C0E7002897DA258695E74E49D4F8DC0047
:1043D000884202D2401CC4F8DC00E07B082803D1EC
:1043E000D4F8DC00884210D33D70A068C10506D522
:1043F00020F0080005E00CE031E02CE034E040F073
:104400000800C4F8DC50A06075E7BDE8F05F02F07A
:1044100015BCE07B092801D025863AE1DBF81C00B9
:104420005F46401CCBF81C00022809DD388D0123B3
:1044300001B2388B052200B200F05AFAFD61B86271
:104440001D48398D44300180B6F844104180FEF794
:1044500061F820864FE7BDE8F05F04F061B82A48B4
:10446000007809287ED046E7284BDFF8A4E01888BA
:10447000401C82B227481A80C82A04D390F800C092
:10448000BCF1010F49D0B2F57A7F04D390F800C097
:10449000BCF1020F41D0B2F5FA6F02D30278032AC1
:1044A0003BD0E07B801E08287DD2DFE800F041AEE3
:1044B000F4F0357C8A04CCE620090020F8060020C0
:1044C000100A00201C0500203C010020980200205A
:1044D000FC060020EF060020D0060020B4080020D3
:1044E0001E000020C6050020F0060020680C0020F9
:1044F000600000209AF9FFFF90090020300C002096
:10450000D28A0008C0D40100540200201600002006
:104510001400002015000020EDE605701D80B9F89C
:10452000062022F40062A9F806208EF80080B8E781
:10453000FDF726FF3078400611D5684880780428BA
:104540000DD0706C82280ADAB07A96F83D1000F02F
:10455000030001F00301884201D001F01FFD38780B
:10456000062800E095E0D7D086F83F50B06C5C4953
:1045700040F31100C86281035A484162FDF7EAFC2A
:104580008BF80780B4F81401A4F81601706CA4F835
:104590008250B0F5437FA4F880A06BDCA16821F4C1
:1045A0008061A16000E092E040F28A21884204DA52
:1045B0003078400601D402F02DFAA06862E038702D
:1045C00099E6706CB0F5437F04DA0878062801D0CC
:1045D0000D7074E04448017821F040010170FDF74E
:1045E000B9FCA4F816A1FDF7CBFE404810F82C1F2B
:1045F00021F0010101703E49C4F8DC504D62394997
:104600004D6208213970456475E699F80600C006C8
:10461000D6D4706CB0F57A7F3BDDFDF7B1FE307813
:10462000400611D52D48807804280DD0706C822862
:104630000ADAB07A96F83D1000F0030001F00301A9
:10464000884201D001F0AAFC2A4886F83F50007841
:1046500010F00C0F03D0B6F84810218602E0B6F82F
:1046600048002086B4F93010514501DDA4F830A08F
:10467000FDF770FCA06840F48060A06096F83810E8
:1046800005299DD140F01000A060022097E713E0BB
:1046900001E03D702FE6706CB0F5437F02DA0878D8
:1046A000062895D1B9F8061021F02001A9F80610C6
:1046B000FDF766FE042082E70878062802D087F816
:1046C000008018E60C4909200870052077E70348A8
:1046D000857003480D7080F8565074E63C04002045
:1046E000600000208C080020FE060020240A002024
:1046F00064080020B40400205402002030B585B0C6
:1047000001210420FFF700FC4FF40040ADF8100039
:1047100048208DF8130004A91848FDF779FD012100
:104720000846FFF7D9FB40F68C20ADF804000324BF
:104730000020ADF80040ADF80200ADF806004FF0E3
:1047400080456946284600F0B9FF1C208DF80C0012
:104750008DF80D408DF80E4001208DF80F0003A854
:10476000FFF79AF801221146284600F081FE012148
:10477000284600F0AFFD05B030BD00000008014044
:10478000704700002DE9F041304CE07800285AD104
:104790002078002857D0401E10F0FF00207052D122
:1047A0004FF49670208272B6294F45F2AA50A7F8AE
:1047B00072000020FDF7ACFB264D13202860FDF7AA
:1047C000B9FBA8BB3420E86002202861224E6E614C
:1047D000286940F040002861FDF7ACFB40BB002198
:1047E0001E4A08465FEA255312F800C0BCF1FF0FCD
:1047F00000D00121401C80B29842F5D3C1B9C4E970
:10480000067639260127A06910F8011B10F8012B44
:10481000A061E06901EB022102886A612F6120F842
:10482000021BE061FDF786FB10B9761EB6B2EAD234
:104830000120FDF76DFB62B601F004FC08488168B9
:1048400021F480418160BDE8F0810000EC06002089
:10485000680C00200020024000FC000800FC00085A
:10486000980200201948016841F0100101600168B8
:1048700021F003010160016841F002010160144868
:104880004168416041684160416841F48061416034
:10489000416821F47C11416041680E4A1143416036
:1048A000016841F08071016001688901FCD54168AF
:1048B00021F003014160416841F00201416041681B
:1048C000C1F381010229FAD17047000000200240A3
:1048D000001002400000280830B5044C039D6080A1
:1048E000A180E2802381658130BD0000040A0020A0
:1048F0000A44824201DA10B27047C91A8142FBDDD4
:1049000008B27047F0B53E48DFF8F8E03E4CC17F92
:10491000467A056800233D4A3D484FF0010C802946
:1049200025D301F01F015EF821100D4201460968F0
:1049300002D041F4805101E021F480510160CF04A4
:1049400011D48F040FD5977AFF0705D053812778AC
:1049500027F00207277006E090F846709FB1012FFC
:1049600014D080F846300F0B67F34D310160802E74
:1049700025D306F01F015EF821100D42016809D011
:1049800041F0040108E080F846C0ECE7022780F817
:104990004670E8E721F0040101604D070BD44D0596
:1049A00009D5957AED0706D05381257825F00205C3
:1049B0002570C0F898308C0864F38A210160917AE0
:1049C000C90718D1134991F86410012913D112496C
:1049D000496C32290DDC017849070AD5018909059E
:1049E00007D4D0F8981047F23054A14204D9A2F865
:1049F0000AC0C0F89830F0BD491CC0F89810F0BD4E
:104A0000CC050020F88F0008C6050020100A002001
:104A100098020020680C00203C01002010B5FCF733
:104A2000A9F90F48018821F0020101800C491831D1
:104A300009880C4A928E1144094A3432118008497F
:104A40000C390A8842F001020A80011D0A884FF6DB
:104A5000ED531A400A80018841F01201018010BD17
:104A60000C0400403C04002006480188491C89B21F
:104A70000180B1F57A7F04D34188491C418000212F
:104A800001807047100700200F4810B5016841F001
:104A90000101016041680D4A1140416001680C4A02
:104AA00011400160016821F480210160416821F416
:104AB000FE0141604FF41F018160FFF7D3FE0549FD
:104AC0004FF00060086010BD001002400000FFF8C9
:104AD000FFFFF6FE08ED00E02DE9F0412F4D28889C
:104AE0004FF00004000629D5FCF7C4FA2C4A2D48E3
:104AF00007231778C8262C49012F22D02B4FB7F84F
:104B000006C0BCF1000F3ED0B0F80CC04CF0080C51
:104B1000A0F80CC0B0F806C02CF4006CA0F806C0D9
:104B2000886820F004008860FC801370CE87002025
:104B30004FF49661401C80B28842FBD32C80BDE8C4
:104B4000F0811B4F97F800C0BCF1010F0FD0BCF1F2
:104B5000020F11D0B0F806C04CF4006CA0F806C0EB
:104B6000886840F00400886005203870DDE7B0F800
:104B70000CC04CF0080C03E0B0F80CC04CF0100C6A
:104B8000A0F80CC0F0E70B4F3C70C78847F40067F3
:104B9000C780886840F004008860C6E7102C014098
:104BA000EF060020100A00209802002020090020B3
:104BB000F00600200D070020704700002DE9F043AB
:104BC0004FF08040018A21F001010182AC48007859
:104BD00000287CD1AB4FF87B002878D1AA48406CE4
:104BE000322874DCA9488068DFF8A4924104A94DFA
:104BF000B9F804004FF0000403D4401CA9F80400E5
:104C000028E1002874D02978012611B1012912D099
:104C100017E14946B0F5BE7FFAD92E70CC718C7180
:104C2000EC702C72287A0A18401CC0B214722872D8
:104C30000F28F7D305E1B9F802204946824201D98D
:104C4000EE7100E0EC7192488A7908300F2A15D293
:104C5000CB79082B0BD2C3F10708EB7912F800C00F
:104C600003FA08F363441354CA79521CCA71CA790F
:104C7000082A03D18A79521C8A71CC7199F80610DE
:104C8000C8460F2973D10D21FCF75EF9A881010AEE
:104C90006970C0B2A87088F8064098F816208A4259
:104CA00065D198F81510814261D198F80BC07A4906
:104CB000032302227948BCF1000F10D0BCF1010F90
:104CC00002D0BCF1020F14D080F86A2000E0CBE0E3
:104CD00091F800C02CF00C0C0CF1080C0FE080F8DF
:104CE0006A6091F800C02CF00C0C0CF1040C06E08A
:104CF000A9E080F86A3091F800C04CF00C0C81F803
:104D000000C098F80C10B6EB111F04D180F86E406B
:104D100087F846400EE0B2EB111F04D180F86E60B8
:104D200087F8466006E0B3EB111F03D180F86E20D0
:104D300087F846200B0717D001F00F01012901D099
:104D4000022915D080F86C602C7198F80D102A7922
:104D500006FA02F30B406B71082A44D2DFE802F036
:104D60000B124319242F363D80F86C40ECE768E0C5
:104D700080F86C20E8E713B180F8704033E080F8E9
:104D8000706030E013B180F850602CE080F8504043
:104D900029E023B180F8656087F8036123E080F89B
:104DA000654087F803411EE023B187F8F54080F89D
:104DB0004D4018E087F8F56080F84D6013E013B1BE
:104DC00080F868600FE080F868400CE013B180F86C
:104DD000666008E080F8664005E013B180F867601F
:104DE00001E080F86740521CD2B22A71082AAED383
:104DF00098F80E102A4A8B0705D587F8F16080F8DD
:104E00006460568104E087F8F14080F86440548182
:104E1000C90702D080F8294001E080F8296098F89D
:104E2000111000F86D1FC2781E48012A1ED001B370
:104E3000012921D04FF48051A0F876101A493C2066
:104E40000870A9F80240A9F80440B9F80210491CFA
:104E5000A9F80210B9F80210B1F5FA7F04D940F2AE
:104E6000F511A9F802102C70BDE8F08344F21C7112
:104E7000E2E74FF40051DFE741F25551DCE7000073
:104E8000EF060020980200203C01002000100140A5
:104E9000500C002088060020B4040020680C00207C
:104EA000100A00201C050020EC0600202DE9F05F10
:104EB000FDF766FA8E4D2888A5F10406C0070AD0D2
:104EC000308820F008003080288820F009002880F1
:104ED00001F0A0FDD9E02888DFF81892DFF81882E9
:104EE000864C80071AD5B9F8001041F00101A9F8E5
:104EF0000010B8F80000804914315030088028882C
:104F00004FF6F95108402880308840F00400308086
:104F1000FFF766F884F83C00BDE8F09F2888784FDA
:104F20004007288871D520F004002880FFF758F842
:104F300094F83C108142EFD1308820F0040030809A
:104F4000FDF7F6FB2078410605D594F84C1094F84F
:104F50003B209142E0D03978400621F002013970BF
:104F600004D5FEF7FDFA97F82F7004E094F83C00A2
:104F7000FDF758FA0746DFF880B140F68C2A0BF1AE
:104F8000180B062F47D294F83800B8423ED0384666
:104F9000FDF7CCF92078C00716D094F83A0094F8C1
:104FA000391000F00302914206D0A17A00F001000E
:104FB00001F00101884215D1FDF722FBFBF726FF26
:104FC000FDF74AFC384689E0FDF71AFBFBF71EFFA8
:104FD000FDF742FC3846FDF733FB207840F0010036
:104FE000207099E7288820F008002880206B81082D
:104FF00001EBD000504515D2B8F800100844ABF8CA
:105000000000308840F0080003E00DE0308820F018
:105010000800308080E7B9F8001041F00101A9F8DC
:105020000010DFE75046E7E70007288831D520F079
:1050300008002880308820F008003080FEF7D0FF7C
:1050400084F83C00FDF774FB387820F002003870DB
:105050002078400604D5FEF783FA97F82F5004E035
:1050600094F83C00FDF7DEF90546062D08D294F8C9
:105070003800A842B5D0FDF7C3FAFBF7C7FE2AE017
:105080002048C18841F04001C180BDE8F05FFDF7D4
:10509000C3BBC006288825D520F0100028803088A2
:1050A00020F01000308097F838000C2802D2401C05
:1050B00087F83800387840F002003870FEF750FA70
:1050C00097F82F50787884F8390094F83800A8427F
:1050D00087D0FDF795FAFDF7BFFB2846BDE8F05FE6
:1050E000FDF7AEBA4EF2BE110840288014E700006A
:1050F0001004004000040040240400403C01002053
:105100003C040020100A00202DE9F04F514F85B0DB
:10511000388820F0010038804E4800261030068084
:105120004D4CDFF838A14FF0010894F85C0042F6CE
:105130003029C10774D072B64948816941F40071C1
:105140008161816941F4806181614FF40040FEF723
:10515000ADFE444D00212846FBF7B6FB0021284652
:10516000FBF7A8FBDFF800B100215846FBF7A2FBD4
:1051700000213E48FCF74CFA2846FBF7C1FC584694
:10518000FBF7BEFC4FF46020CDE902068DF8056008
:1051900000968DF810808DF8048069462846FBF74C
:1051A00041FD01231A460F212846FBF78CFD012102
:1051B0002846FBF77FFB00204946401C80B288420E
:1051C000FBD328462E600121FBF7BCFD2868800731
:1051D000FCD524484C30006894F85C1021F00101A3
:1051E0002144A1F85000FBF779FB62B6FEF7C4F842
:1051F00047F69061AAF8001094F85C00401CC0B219
:1052000084F85C000C2822D212491431A1F80080E5
:10521000388840F00100388005B0BDE8F08FFFE726
:10522000134920F00100085A12490880114945F637
:105230005800083908800F4847F25801001F0180C4
:105240000C4920200C390880AAF80090D4E70320EC
:10525000A070E1E7000800403C0400202C0800405A
:1052600000100240002401400028014008000240D4
:10527000B48B0008202C01400029018802D041F0A5
:10528000800101E021F080010180704710B50A889B
:105290004B88CC881A438B8823431A430B891A43C3
:1052A0004B8989891A430A43A0F8442010BD002184
:1052B000018041808180C18001814181818170476D
:1052C0000029818802D041F0010101E021F00101B3
:1052D000818070470029018802D041F0010101E07E
:1052E00021F0010101807047002930F8441F02D0ED
:1052F00041F4004101E0C1F30E010180704700005C
:105300004B4910B5884202D10121C41486E0B0F1A6
:10531000804F09D0474988420DD101210220FEF774
:10532000E7FD0021022064E001210846FEF7E0FDD0
:10533000002101205DE04049884206D1012104207E
:10534000FEF7D6FD0021042053E03C49884206D1F7
:1053500001210820FEF7CCFD0021082049E0384952
:10536000884206D101211020FEF7C2FD0021102045
:105370003FE03449884206D101212020FEF7B8FDE4
:105380000021202035E03049884202D10121441417
:1053900044E02E49884202D10121CC043EE02C4950
:1053A000884202D101210C0538E02A49884202D105
:1053B00001214C0532E02849884206D101214020D4
:1053C000FEF796FD0021402013E02449884206D1D3
:1053D00001218020FEF78CFD0021802009E020497A
:1053E00088420AD1841501212046FEF781FD002163
:1053F0002046BDE81040FEF77BBD1A49884202D125
:1054000001210C040AE01849884202D101214C0410
:1054100004E0164988420AD101218C042046FEF797
:105420007FFD2046BDE810400021FEF779BD10BD8C
:10543000002C01400004004000080040000C004027
:10544000001000400014004000340140004C0140B6
:10545000005001400054014000180040001C004072
:10546000002000400040014000440140004801404D
:10547000002A828901D00A4300E08A438281704772
:1054800030B5028C22F001020284028C8388048BE6
:1054900022F0020224F073050C882C430D89154379
:1054A0004A882A43114DA8420BD0114DA84208D07A
:1054B000104DA84205D0104DA84202D00F4DA84271
:1054C0000DD122F008054A8923F440732A4322F0C3
:1054D00004058A882A438D891D43CB892B43838009
:1054E0000483C9888186028430BD0000002C0140FD
:1054F00000340140004001400044014000480140A8
:10550000028B22F008020A430283704770B5028CB6
:1055100022F010020284028C8488038B0D8823F40D
:10552000E6464FF6FF7303EA052535430E8922F060
:10553000200203EA061616434A8803EA021232439F
:10554000104EB04202D0104EB04215D122F080066B
:105550004A8924F4406403EA0212324322F04006EE
:105560008A8803EA021232438E8903EA86062643BA
:10557000CC8903EA8404344384800583C988018785
:10558000028470BD002C014000340140028B4FF6B4
:10559000FF7322F4006203EA012111430183704783
:1055A00070B5028C22F480720284028C8488838B12
:1055B0000D8823F073031D4322F400730E894FF608
:1055C000FF7202EA06261E434B8802EA0323334396
:1055D000104EB04202D0104EB04215D123F40066F6
:1055E0004B8924F4405402EA0323334323F48066B6
:1055F0008B8802EA032333438E8902EA0616264388
:10560000CC8902EA0414344384808583C988818765
:10561000038470BD002C014000340140828B22F0D5
:1056200008020A438283704770B5028C22F48052CC
:105630000284048C8288838B0D8823F4E6464FF61F
:10564000FF7303EA0525354324F400560C8903EA69
:10565000043434434E8803EA06362643094CA042FC
:1056600002D0094CA04205D122F480448A8903EA81
:105670008212224382808583C988A0F84010068464
:1056800070BD0000002C014000340140828B4FF6B9
:10569000FF7322F4006203EA012111438183704702
:1056A000018582827047828822F07002828082881F
:1056B0000A4382807047A0F84010704730B50288D6
:1056C0001B4B1C4C98420DD0A0420BD0B0F1804F28
:1056D00008D0194DA84205D0184DA84202D0184D47
:1056E000A84203D122F070054A882A43154DA842EA
:1056F00006D0154DA84203D022F44075CA882A432B
:1057000002808A8882850A88028598420AD0A0424F
:1057100008D00E4A904205D00D4A904202D00D4A60
:10572000904201D1097A01860121818230BD0000B9
:10573000002C0140003401400004004000080040FB
:10574000000C0040001000400014004000400140E8
:1057500000440140004801404FF6FF718180002164
:105760000180C1804180017270470029018802D008
:1057700041F0020101E021F002010180704700299F
:10578000018802D041F0040101E021F00401018010
:1057900070470000204810B590F82010026801F012
:1057A0001F001E4951F820001D490242086802D01E
:1057B00040F4803001E020F48030086019484FF058
:1057C000000280794106184824D4184903880C88BF
:1057D000E31A9CB201230F2C08D30C880480846840
:1057E000042C03DD124C2478022C05D0427F012AC0
:1057F00006D00988418010BD4377C2770A8842806D
:1058000042880988891A89B240F21A629142F2D319
:10581000C37710BD427710BDCC050020F88F00087B
:1058200098020020100A0020300C0020F80600200A
:10583000EF0600202DE9F04FDFF8B8B16A48DFF835
:10584000AC91DFF8ACA190F80EC0BBF91A70BBF9AF
:105850001C60BBF91850BBF96C10BCF1070F48D2A3
:10586000DFE80CF08D041A30485E7600D9F800208D
:105870008284DAF80020C284828CC38CA7EB820277
:1058800012B2A6EB83034A431BB2594342F3CF2221
:1058900041F3CF23D11870E0D9F800204284DAF820
:1058A0000020C284428CA5EB820213B2C28C4B430F
:1058B000A6EB820212B243F3CF24514341F3CF232C
:1058C000E11814E0D9F80020C284DAF800204284FC
:1058D000C28C438CA6EB820212B2A5EB83031CB2EE
:1058E0004A43614342F3CF2341F3CF24191949427C
:1058F0000AB244E0D9F800208284DAF80020428419
:10590000828C438CA7EB820212B2A5EB83034A433D
:105910001BB2594342F3CF2241F3CF24111914E0B3
:10592000D9F800204284DAF800208284428C838CEB
:10593000A5EB820212B2A7EB83034A431BB242F3E8
:10594000CF24594341F3CF22A11849420BB216E0AC
:10595000D9F80020C284DAF800208284C28C838CBB
:10596000A6EB820212B2A7EB83031CB24A4342F3B6
:10597000CF23614341F3CF22991849420CB2BBF9BE
:105980001E50594605F21E56A64201DACE8306E0A5
:10599000A5F21E55A54201DDCD8300E0CC83B1F90F
:1059A000204004F21E55954201DA0D8406E0A4F26F
:1059B0001E54944201DD0C8400E00A84B1F92220D7
:1059C00002F21E549C4202DAABF8224008E0A2F236
:1059D0001E529A4202DDABF8222001E0ABF82230E1
:1059E000417B8173BDE8F08F980200203C24014088
:1059F0003C2801401C0500202DE9F04704465C4886
:105A00005D4D002602785B48022AB0F9301004D0C0
:105A1000082A70D0092A6FD0A5E0C27B022A02D1E1
:105A2000B0F840204AB1E18769810423B5F9081034
:105A30001A460020FEF75CFF8CE05049DFF84081F9
:105A4000496A0F14E7808068410210D5B4F902005A
:105A500040F2DA21884269DD40F26A4188423FDC47
:105A6000A0F2DA20FAF7DBFC0022464B4DE0C0F34F
:105A7000C001C0F30020DFF8109181420CD1D8F8AA
:105A8000440040F2BA41884250DD40F66A11884233
:105A900026DCA0F2BA4034E03C480078C0060CD5C1
:105AA000D8F8440041F2243188423FDD41F2D471FC
:105AB000884215DC00F6DC4021E0354890F8701093
:105AC000012903D090F86F0001282FD1B4F902000A
:105AD00041F6C811884229DD41F6786188420CDD23
:105AE0000823B4F93E101A460020FEF701FFE087B4
:105AF000002819DB1BE02FE033E000F5C760A0F5BC
:105B00000050FAF78CFC00224B46FAF7F4FB0E2209
:105B1000FAF760FCFAF7BAFC00B2C0F580407843AF
:105B20008013E087002F02DCE68700E0E787E08F44
:105B3000184FE880D8F844107964A7F84C0000F0BA
:105B40007DFBB7F84E00688198F80A000028388F6E
:105B500000D14042288106E00F48B0F87400688107
:105B600000E069812E8184F83C60BDE8F087000088
:105B7000EF06002098020020600000201C05002095
:105B80003C0100200000794000C09240D006002077
:105B9000680C0020B4080020240A00202DE9F04100
:105BA000B1F9025000232B241522854203DAB1F902
:105BB0000000BDE8F081B1F9AE50854202DDB1F9D7
:105BC000AC00F6E701EB8205B5F90250854201DD34
:105BD000134600E01446E21852085D1CAA42F1D1B7
:105BE00001EB8206B6F90230834206DA36F9025C2E
:105BF00036F9044C31F9221006E01D4631F92240F5
:105C0000B6F90630B6F90410401B091BC6178911F6
:105C1000B60346EA90468703A1FB070CCA1702FBAE
:105C200007C201FB06215A1BD317FAF77DFA000AB7
:105C300040EA0160001900B2B0F5804FB9DB43F6CD
:105C4000FF70B6E770B5134C40F224452946204654
:105C500000F03EF800281BD0204600F0C7F8294687
:105C6000204600F01DF80C4C00212046FBF7D0FC2C
:105C70002046FBF74BFDC0F164000849C0B2042880
:105C8000087201D900F046F9BDE87040FBF784BD09
:105C900070BD000000380140580002405806002046
:105CA0000A0A01219140C943018070470029818976
:105CB00002D041F4005101E021F40051818170478C
:105CC000002A828A01D00A4300E08A438282704718
:105CD00030B501F01F0201240025C1F3421304FA7C
:105CE00002F2012B0FD0022B0FD0838A4FEA112131
:105CF0000088134204FA01F400EA040001D000B164
:105D00000125284630BD8389F0E7038AEEE710B508
:105D1000C1F3421301F01F040121A140012B07D060
:105D2000022B07D01430002A026805D00A4304E091
:105D30000C30F8E71030F6E78A43026010BD00002F
:105D400030B50446008A85B00D464CF6FF71084018
:105D5000E98801432182A1894EF6F3100140A88809
:105D60002A8910436A890A431043A081A08A4FF60A
:105D7000FF410840A9890143A1826846FEF7DCF88B
:105D80001948844201D1039800E00298A1890904CE
:105D900000EBC00101EB0010296801D5490000E0CB
:105DA0008900B0FBF1F06422B0FBF2F109010B09AC
:105DB0006FF018056B4300EB8300A3891D044FF0BF
:105DC000320306D503EBC000B0FBF2F000F0070091
:105DD00005E003EB0010B0FBF2F000F00F00084309
:105DE000208105B030BD0000003801408088C0F33C
:105DF00008007047F8B501210920FEF785F8012158
:105E00008803FEF781F810258DF803502020ADF8A7
:105E100000001A4E03248DF8024069463046FCF714
:105E2000F7F916490C31086820F0200008601820A6
:105E30008DF803004020ADF800008DF8024069465F
:105E40003046FCF7E5F948208DF803008020ADF8D6
:105E5000000069463046FCF7DBF98DF80350280155
:105E6000ADF800008DF8024069463046FCF7D0F9E5
:105E700001210420FCF71EFAF8BD0000000C0140CF
:105E800030B585B0FFF7B6FF00244FF4E130009045
:105E9000ADF808400C201D4DADF80440ADF80A00E7
:105EA000ADF80640ADF80C4069462846FFF748FFBC
:105EB00025208DF8100004208DF811008DF8124077
:105EC00001208DF8130004A8FDF7E6FC012240F242
:105ED00024412846FFF71BFF01212846FFF7E6FE75
:105EE000FBF784FC012280212846FFF7E9FE01220E
:105EF00040212846FFF7E4FE012202210448FBF777
:105F000019FCFBF773FC05B030BD00000038014000
:105F10004400024070B51D4D00242878432834D138
:105F20006878462831D1A878502807D0512805D064
:105F3000812803D0892801D0212826D1144E7071E0
:105F4000E9787172A81C891CFBF736F8B072717A77
:105F5000294409793182884217D106F10E0001786F
:105F600041F0020101700B48016841F0200101601D
:105F7000317A0948002204E02B5D03552A55641C40
:105F8000E4B28C42F8D38078707170BD8407002031
:105F9000580600200C0C01409A0B002070B51D2003
:105FA000FDF759FCFDF7DCFA1D20FDF76AFC1548EA
:105FB00090F82F10144D0623144C85F8381090F8E3
:105FC0003B1095F83B201143012A04D0022A07D048
:105FD000042A0AD010E0827A8A420DD0007B09E0C0
:105FE000027D8A4208D0807D04E0827F8A4203D00D
:105FF00090F82000884200D12370002085F84000EE
:1060000070BD00003C0400203C010020EF06002091
:106010000B4800214180A0F1B0018A898280CB89A0
:106020001A44C2800B8A1A4402814B8A1A44428164
:10603000898A1144818143F6FF71C1817047000054
:10604000EC010020084940F61C72B1F90C009042A6
:1060500002DA00F59F7005E041F2E302904201DDB3
:10606000A0F59F70C88170476000002038B51348C4
:10607000C16941F00401C1611E208DF800000220B9
:106080008DF801008DF8020001248DF80340684668
:10609000FDF702FC0A4984200880094947F6906010
:1060A0002C3108800020091F0880054914310C801C
:1060B000091F0880081F048038BD0000001002403E
:1060C0000008004030B420491E4A45788B7A1146BA
:1060D00092F83B4091F83910AC4218D14BB103799A
:1060E000994202D04379994201D140791AE08079EE
:1060F00009E08379994202D0C479A14202D182F8A1
:106100002F3011E0407982F82F0030BC7047C578FD
:10611000AC42FAD16BB1C379994202D0037A994269
:1061200005D1007A82F82F0030BCFEF777BC407AA8
:10613000E9E7437A9942E2D00479A142DFD0007ABC
:10614000E1E700003C0400203C010020FEE70000E5
:106150002DE9F0470446007F012868D13548E188E1
:106160000288511A89B2072916D30088E080B4F951
:10617000000044F2DD414843401346F6D9614843EC
:106180008013A060401000B2A0814FF08051B1FB9D
:10619000F0F0FAF73FF92061B4F90C6096B1B4F968
:1061A00002104DF6B05048430014A082B4F90470B8
:1061B0004DF6B05207FB02F24FEA2245E58204D4C5
:1061C000024603E00020E08330E0424212B2228324
:1061D000002D01DB2B4600E06B421BB2DFF858902C
:1061E000638398464FF4804AB24208DAFAF709F915
:1061F0002169F9F7DCFFFAF730F9801304E0002990
:1062000001DA484600E05046E083B04509DA284606
:10621000FAF7F7F82169F9F7CAFFFAF71EF98013C0
:1062200004E0002F01DA484600E050462084BDE833
:10623000F0870000F806002000C0FFFF10B52848D6
:10624000294C01782748022905D1C17B022902D1B6
:10625000B0F8401029B1008EA4F84E00002020872D
:1062600010BD90F8462020482049022AB0F844008A
:10627000097800B2C1F3810103D0012A0CD01C4976
:1062800013E0012904D0022904D019496C390CE02B
:1062900018490AE0184908E0012904D002291CD055
:1062A00015496C3101E013496C31FBF701FE0E49D1
:1062B000A4F8400080B2483101F060FAB4F94C0013
:1062C000B4F94A2041425143891324F8381FB4F9E4
:1062D000101048438013E08210BD07496C39E4E791
:1062E000EF06002098020020B4080020B40400202B
:1062F000488A0008C0870008048900080348002174
:1063000080F82A10C183018770470000B40800207C
:1063100010B504000B462D4AC3F1000028D5644295
:10632000002B12DAA04207DA214600F027FA32F8F1
:106330001000C0F5404041E00146204600F01EFA42
:1063400032F8100000F5004038E0A34208DA214698
:10635000184600F013FA32F8100000F540402DE026
:10636000204600F00BFA32F81000C0F5803025E02E
:10637000002B12DAA04207DA214600F0FFF932F8CA
:10638000100000F5804019E00146204600F0F6F9C3
:1063900032F81000C0F5004010E0A34208DA2146B0
:1063A000184600F0EBF932F81000C0F5804005E027
:1063B00053B1204600F0E2F932F81000B0F5004F7A
:1063C00001DDA0F5803010BD002010BDC08B00089D
:1063D00040438013494300EBA13000220302002B0D
:1063E00014DDB3F5001F01DC802001E04FF4005004
:1063F00093FBF0F1014401EBD1714910814206D0C9
:10640000521CD2B20846062AF2D300E00021C8008E
:1064100000B2704702E008C8121F08C1002AFAD172
:1064200070477047002001E001C1121F002AFBD114
:10643000704700002DE9F047A44CA5482188028848
:10644000511A89B20F297DD30088A4F13C05208020
:10645000288F08B1401E28872B789E4AC3F38100FD
:1064600001281DD0022820D0D18B98489A4FDFF800
:106470006C92407E0026B1F5926F1DD8142819D376
:1064800078206076F88840F01000F88040F266606E
:10649000A88123F001002870D67389F8006015E008
:1064A000D08B00EB4000C00302E0D08B8C49484306
:1064B000010CDAE7401C04E0B1F5DB6F06D310B144
:1064C000401E607602E043F001002870B5F902003A
:1064D000B5F914304143C3EBC303C1F38F31C3F3A8
:1064E000D10303EB510109B2A9829046D28B4FF040
:1064F00080535043B5F91620C0F38F30C2EBC2026F
:10650000C2F3D10202EB500000B2E882AA6A424311
:106510001213EA6293FBF2F22A63724A1080A268B5
:106520000A44A260E1680144E160207C401CC0B2E2
:106530002074072806D942F3CF002883C910698345
:10654000E66000E0BFE0A66041F6C801267488421C
:1065500004DD298B644AB2FBF1F1E981C11789039B
:1065600041EA9041800342F69B420023F9F7DCFDAB
:10657000A88456482A78A0F13C005C49B0F906008E
:10658000930700FB01F14FEA2141C2F3810215D5C7
:10659000012A07D0022A0BD04FF268514143091457
:1065A000A18011E049F68C4250430014A0801FE006
:1065B0004CF6183141430914A18025E0012A0DD081
:1065C000022A17D0A0806984494948430014E08317
:1065D000FBF78EFA47480088C0B143E04AF65C32C8
:1065E00042431214A2804BF62C22504300146884BC
:1065F000E183EDE74DF2AC5141430914A1804EF225
:106600007C414143091469843B49DEE795F8200049
:1066100000BB88F80F6089F80060B5F91A00A0F592
:106620000C519F39B1F56E7F18D8617FF42912D9CA
:106630003249E8802E4AA1F8460050430014A88051
:10664000A1F84400FF2085F8200081F828002C499B
:106650003C20087006E0491C617703E0607F08B1C8
:10666000401E6077B5F91A10B4F91E0081420EDDA4
:10667000A07E7D2809D9F88840F00800F8802148DC
:10668000017821F0020101700EE0401C06E0A0F24A
:106690003D10814208DAA07E10B1401EA07603E0D2
:1066A000F88820F00800F880B5F9181060690844EF
:1066B0006061217E491CC9B221761F2903D940118E
:1066C000A88366612676BDE8F0870000F00400200C
:1066D000F806002098020020100A0020EF06002093
:1066E00030330100C409002074E8260BCC0E0100F1
:1066F00048850100FA060020D0450100680C002002
:10670000EC060020C6050020024941F68B30886265
:1067100070470000B404002070B5164C06252078A0
:10672000062825D2DFE800F003080E141A211248CB
:10673000FAF780FC012016E00F48801DFAF77AFC7A
:10674000022010E00C480C30FAF774FC03200AE039
:1067500009481230FAF76EFC042004E006481830AD
:10676000FAF768FC0520207070BDFAF783FC2570ED
:10677000257070BDF0060020B48A0008090A05D013
:10678000B0FBF1F0FF2800D9FF20704700207047D0
:10679000D0E90021C368521A5A4301EBA23181604B
:1067A00041607047B0F90020B0F90210B0F906302E
:1067B000521A5A4301EBA231818041807047000098
:1067C00030B5444B188844498A89801A85B24348B9
:1067D000434A0F2D047801F14C001DD31D888D8193
:1067E000117A090713D5022C01D03E4912E03E4D23
:1067F000B0F90210B5F90050A94205DC02DA01F146
:10680000020108E0458007E0A1F1020103E0022C4B
:1068100002D1364909884180018F1D88691A89B2E1
:106820009C2942D319880187916A0023B1F5804FD2
:106830002DDB2F49896CB1F5405F28DD2D4940F2F1
:106840006665B1F91010A94211DD43F69915A94208
:1068500002DB40F2333108E040F23335A1F26661E9
:10686000694343F2333591FBF5F1818700E083877B
:106870002149B2F806510978C1F381011DB1818F18
:1068800001F21E5119E092F84620022A0ED08387A9
:10689000022C00D08387B0F95410B0F93C3001F1DC
:1068A00014029A420BDAA0F8542030BD012901D01D
:1068B0000229E4D1818F01F233318187E8E703F1C6
:1068C0001402914203DD1439A0F8541030BDA0F831
:1068D000543030BDF806002014000020EF060020E0
:1068E00098020020B2040020B0040020AC04002074
:1068F0003C0100201C050020B40400202DE9FC41CF
:1069000001210220FDF7E8FA01211920FDF7FCFA28
:1069100001213C48FBF7CEFC4027ADF80070032472
:106920008DF802400420384D8DF803006946284652
:10693000FBF76EFCE001ADF800008DF802401C2072
:106940008DF8030069462846FBF762FC4FF4E071BE
:106950002846FBF7E4FCA815ADF800008DF80240CE
:1069600010208DF8030069462848FBF751FC4FF4CE
:10697000A060FCF7C3FF1D208DF8040001268DF8F0
:10698000056000258DF806508DF8076001A8FCF71A
:1069900083FF1F498C2008801D494FF6FA702C3167
:1069A00008806E20091F0880194814300680184896
:1069B00008300780164920310D80154AD020121D5D
:1069C0001080134A45F2F300183210800A1F45F276
:1069D000500010800E4A4FF6FF7038321080121DA2
:1069E0001080121D108041F21B10088000F012F878
:1069F000FBF712FF064810300580001F0480BDE839
:106A0000FC810000000C1A0000100140000C014045
:106A10000004004070B51D20FCF712FF2A4D4021F4
:106A20002846FBF773FC840080212846FBF76EFCA8
:106A300044EA4004A9152846FBF768FC0443E0B289
:106A4000224C84F83C00FBF7EDFC0546052805D9EF
:106A50001F48C18841F04001C18001E084F83850EE
:106A60001C48007A000703D594F838001A490D5CD9
:106A70004FF6FA702063E062A06260622062E0611B
:106A8000A0611648606300206064A06484F83F0041
:106A900084F84000FBF774FCA07AFF2811D0022094
:106AA00084F83D000E48008820662846FCF716F959
:106AB000207820F001002070BDE870401D20FCF718
:106AC000D5BE0120ECE70000001001403C01002091
:106AD000100A002098020020C4930008DCFF050083
:106AE000240400402DE9F0434E484F4902880B88AA
:106AF0009A1A92B20F2A69D3098801804B49098BEF
:106B0000027D00EB42029180017D491CC9B20175F2
:106B100008295BD3002404752246017D00EB410364
:106B2000491CB3F90430C9B202EB630212B2017519
:106B30000829F2D33E4904753E4B4A8044800E78C2
:106B40009D895FEAC67C40F638694FF0030714D090
:106B5000A2F22B5C42F6E858C44520D3A1F1020C06
:106B600026F00204ACF8002047750C7040F22B545C
:106B7000A24211DA45F004021EE046F001060E7052
:106B80004A4507DD45F001029A8126F002020A70AB
:106B9000477519E0447517E045F002020CE04A45DC
:106BA0000CDA8775427D12B1521E42750CE046F038
:106BB00002020A7025F007029A8105E0B30703D5A7
:106BC000837D2BB15B1E837540888880BDE8F08390
:106BD00042F6AA239A4222DAB1F904302BB941F2E3
:106BE000CD05AA4201DA4480EEE7134C920302EB92
:106BF000843241F67244B2FBF4F214B240F23335FF
:106C000002464480AC4200DA5580B2F90240E41AF0
:106C100004F5A374B4F5237FD6D84380D4E74FF4AA
:106C20008043FAE79C0A0020F80600209802002022
:106C3000C6050020100A0020C8F1FFFF2DE9F04131
:106C40006C4CDFF8B4E14FF0000594F82C10C80745
:106C500006D094F930104B42002956DD0E4655E01F
:106C6000664884F82F506587654A90F8380084F8A4
:106C700038001586CEF80450CEF80850614E40F228
:106C80006663CEF80C50A4F8743036F810005E4EEF
:106C9000768830444FF6FF7606EA800024F8280B09
:106CA0004FF080602060A320208460845810A0846E
:106CB000E38440F699102085580060854FF4805099
:106CC000A08541F23330E08541F26660208641F6CE
:106CD0009910608641F6CC40A0864FF40050E086C3
:106CE00042F23330208742F26660608742F69910A4
:106CF000A08742F6CC40E08782F89D5041F0010029
:106D0000207184F84450BDE8F0811E4694F92F00AC
:106D10004242002801DD074600E01746F61B012E1F
:106D20000BD0002800DB02465FFA82F684F83000C0
:106D300094F84700012805D041E0002900DA1946FF
:106D4000CEB2F3E794F931305942002B01DB1846FB
:106D500000E0084694F93220C7B25042002A01DB15
:106D6000944600E08446BC4508DD002A00DA02466D
:106D7000D7B2002B00DA0B46D8B207E0002B00DABE
:106D80000B46DFB2002A00DB1046C0B204EB400025
:106D9000B0F9481004EB470030F9482F114449106E
:106DA000018084F8475084F8365084F8355084F8D0
:106DB000345084F8335084F8325084F8315004EB66
:106DC00046007546B0F948006087BEF80410C82335
:106DD00009B26422FDF78CFD6860E968401AA96871
:106DE0000844A860B5F900104843C013E860A4F84F
:106DF000740088E7240A0020B40500203C0100202C
:106E000098020020D693000860000020F0B4544897
:106E100090F82C10C90776D0524990F838300022EB
:106E200091F838108B426FD04F4CA0F86A204F4D2C
:106E3000E65C04468E4294F92F4002D0EE5C8E420E
:106E40000FD1641C64B280F82F40EB5C8B4202D1FE
:106E5000641C80F82F4090F92F300F2B1BDD0F237F
:106E600017E0434DEE5C434D8E4202D0EE5C8E4205
:106E700011D1641E64B280F82F40EB5C8B4202D1CA
:106E8000641E80F82F4090F92F406FF00E039C4253
:106E900001DA80F82F30324B90F83750313390F8C8
:106EA0002F40EC5490F837305B1CDBB280F8373061
:106EB000062B01D380F8372090F9314090F9333018
:106EC0009C420ED190F93540A3420AD190F932404C
:106ED00090F934309C4204D190F93640A34200D15D
:106EE000012280F847201F4A80F8381090F92F506F
:106EF0001378214A012D0DDD14465E07A46804D5E0
:106F000044F0080403E028E015E024F0080494604D
:106F100080F82D10B5F1FF3F0ADA5B07936802D5C0
:106F200023F0080301E043F00803936080F82D107C
:106F3000F0BCFBF725BA90F8471001290DD1B0F845
:106F40006A1043F60953491C89B2A0F86A109942A5
:106F500003D9A0F86A2080F84720F0BC70470000F1
:106F6000240A00203C010020B8930008BE930008CA
:106F7000CA930008D09300089802002030B5204939
:106F8000204AB1F86A301088C01A80B20F2836D370
:106F90001088A1F86A001C4D00204FF000432A5CC5
:106FA000940903D00124B4EB921F24D1D20622D03D
:106FB000164A52F820201268134C123434F810404C
:106FC000224201EB000494F9722008D00A2A04DB63
:106FD0000A6823FA00F4224308E0521C09E012F187
:106FE0000A0F05DC0A6823FA00F4A2430A6002E0F3
:106FF000521E84F87220401CC0B21128CFD330BD7D
:10700000CC050020F8060020C48F0008C4900008BA
:107010002DE9F00779497A480A8903889A1A92B2C9
:10702000082A74D300880881A1F12C0042890AB192
:10703000521E4281734A92F82820802A67D302F0B8
:107040003F020A70C2890AB1521EC281B1F90620FC
:10705000902A0CDB8A46FF2A09D08146C089002885
:1070600055D1694800230078092805D005E0BDE81E
:10707000F007624800F092B90823644A92F8EA5097
:107080000DB143F004036248817AC90701D043F08F
:107090000203D2F808C05FEA0C5101D543F00103A6
:1070A000176800215B4EFC0302D596F8654004B1D9
:1070B0008021C4885FEA446801D541F040015FEA5D
:1070C000845801D541F020015FEAC47801D041F035
:1070D0001001007A400701D541F008014E480078C0
:1070E000C00701D041F00401A00601D541F0010123
:1070F0000020012D00D1082096F8705085B992F833
:107100004620022A04D0012A05D03AB108E072E0F4
:1071100040F0030004E040F0020001E040F0010014
:107120007A0701D440F02000CCF3C0020025CCF354
:10713000002C624502D13A0700D4042596F86F204E
:10714000012A01D145F00105344A0027BC461278D6
:107150003E46C2F38102012A04D0022A04D0032A47
:1071600004D004E0022602E0042600E010262C4AA7
:1071700064060ED5214C1C342478240609D51478D5
:10718000640606D4274A40F6CC44926D6243140C40
:1071900005E0B2F8AE2040F699146243940B4FF02C
:1071A00008088AF80A804FF061088AF80B808AF88C
:1071B0000C308AF80D108AF80E008AF80F508AF801
:1071C0001070270A4B4083F06901414069408AF8FA
:1071D000117079408AF81240614052468AF813C013
:1071E00071408AF8146051754FF4C871A9F80E10F7
:1071F000FF20AAF80600BDE8F0077047B40600209B
:10720000F8060020CC050020EF06002098020020A0
:10721000100A0020680C002008090020B404002097
:107220003C010020E80700204C48816941F0FC0146
:1072300081614FF4A060FCF761FBFBF77BFBFCF77F
:10724000C1FCF9F7B5FCFCF7B7FAFDF757FAFFF701
:1072500055FBFCF7F7F9FFF7DDFBFBF7DDFA404DD7
:107260004FF40050A5F81601FEF70AFE00214FF476
:10727000FA5340F2EE220020401C80B29842FBD329
:10728000491C89B29142F6D33648002680F87260D4
:10729000F9F724FBF9F7CAFFFCF7C4FCF9F798FEED
:1072A000FEF7E4FE102230493048F8F76EFF304C0C
:1072B000314FE08820F04000E0802E48017821F036
:1072C00020010170FA20F8814FF49670E887FFF7EB
:1072D0001BFA2A492A48FCF722FC2A48FCF744FCFE
:1072E0002948416A88472948416B8847FFF706F8D3
:1072F00027494220C8802749C8603E71E088E08164
:107300002089208260896082FAF7FAFEFAF75CFE33
:10731000FFF790F8FFF7E6FB00F0F8F9FFF72EFE15
:1073200000F0C2FFFEF736FAFAF7B2FCFBF7F4FC06
:10733000FFF746FAFCF7CEFEFBF716F9FBF748F924
:1073400000F07AF8FFF764FE1348FAF799FA00F0B4
:107350006FFAFDF717FAFAF7FDFBCFE700100240CE
:10736000980200201C050020680C00200C0600205C
:10737000100A00203C010020EC0600208C080020B0
:1073800064080020F803002034000020D000002012
:10739000140700202804002090090020F0B523499C
:1073A0000278B0F9064000231F4E31F81210FF2C6E
:1073B00018D0B0F904701E4DBC4231DA00EBE4077E
:1073C00004F00704BF7AA7408478FFB23CB190F87C
:1073D00001C0ACF1010C64451FDA3C061DD455F820
:1073E00022200DE056F82220116012498A79521CA1
:1073F000D2B28A71022A02D38370C3808B71F0BD2E
:1074000011608178491CC9B2817042789142F6D3EB
:107410008370C188491CC180F0BD56F82220EFE777
:1074200055F822201160F4E7A4910008D68F0008D7
:107430004C91000888060020F0B561486149B0F819
:107440006C200B889A1A92B29C2A7BD30988A0F8E8
:107450006C105D495D4F91F82A1001F0070297F812
:107460004610022A00D1491E594C80F83E104FF0B8
:107470000203E2884FF00001550401D5012236E0F5
:10748000A489E50601D5062231E0250701D50822A9
:107490002DE0550603D44F4D2D78AD0601D50422BD
:1074A00025E0150501D5072221E0150601D50A22A0
:1074B0001DE0950601D50C2219E0150701D50B2218
:1074C00015E0550701D4D50501D510220FE0D506EA
:1074D00001D505220BE0650703D4A50701D4E40715
:1074E00002D080F86E3007E0920403D5032280F8C2
:1074F0006E2001E080F86E10374A384C92F820E098
:10750000324A251FD2F808C02D4AB2F87060721CAA
:1075100092B2BEF1000F0DD02CF4000CC7F808C0D9
:1075200090F86E70B7B11E2F1AD090F86F200AB382
:1075300025E007E04CF40006BE60A0F870200A2A9F
:1075400001D22360F0BD142A01D22B60F0BDA0F857
:107550007010F0BD2B60A0F8701080F86F10F0BDB7
:10756000642E04D2A0F87020322AEED3E9E7A0F806
:107570007010EAE77F1C80F86F70A0F8701090F828
:107580006F20012A10D0002AE9D0B0F87060761C74
:10759000B6B2A0F870601E2ED7D323603C2EDED981
:1075A000521E80F86F20D2E7B0F87020521C92B2C1
:1075B000A0F870202360C82AD1D980F86F10C6E7E0
:1075C000CC050020F8060020680C0020980200205E
:1075D000100A00203C010020B4040020141C0140CB
:1075E000F0B54248B0F84810491C89B2A0F84810DC
:1075F00002297AD33E490024A0F848400A783D4B3E
:10760000042A57D04FF48041082A0BD0A0F10C0275
:10761000B2F900208A4200DA1146B3F980208A428A
:1076200000DA1146344A92698A4200DA11B2418284
:1076300082881D8AC2EB8502304D12B22D78C5F3C7
:1076400081062A4D42F2AA467243B5F9765092124B
:107650006A431213C26086681546C6EBC60642F33B
:10766000D102F60202EBA6328260C66C1644C664F2
:10767000B0F850707F1CBFB2A0F85070B7F5806FA3
:1076800004D3B6120682A0F85040C464891A1C4E76
:10769000C26A724340F255564E4302EB4602466AB6
:1076A00032444262B3F93030B2EB034F06DD1A04C4
:1076B000426206E01349B1F90410B3E7002A00DA88
:1076C0004462C162104990F83D2091F838108A4216
:1076D0000BD080F83D10B0F84210A0F84410B0F87C
:1076E0004010A0F84210A0F84050F0BD1C0500204A
:1076F000EF06002098020020000C0020B4040020B7
:10770000C3F5FFFF1C0C00203C010020174818495E
:10771000B0F85A200B889A1A92B20F2A25D30988FA
:10772000A0F85A10134941F6515391F84D10CA0769
:1077300001464FF48042B1F9001059438913A0F873
:107740006C100D490B78A0F10C01022B06D1B1F998
:107750000030934202DA1B1D0B8000E00A800021FA
:10776000A0F8601020F85C1F428070471C050020C4
:10777000F8060020680C0020EF0600204FF6FF728C
:1077800002EA800210F4404315480ED0B3F5804F52
:1077900014D0B3F5004F4FEA122216D0C2F5807311
:1077A00030F813305B424B8005E0120A30F812309B
:1077B0004B80C2F5807230F812000FE0120AC2F559
:1077C000807330F813304B8005E030F81230C2F58A
:1077D00080725B424B8030F8120040420880704754
:1077E000C08D0008104A518A908AD28A16384639CC
:1077F000A2F1110200D54942002A00DA5242114496
:10780000002800DA40420844084943F6284300B201
:10781000B1F936205A43921340F2D733584302EB62
:10782000A030C88670470000980200201C05002088
:10783000F0B5904990480A8903889A1A92B23E2A74
:107840001ED30088088101F138004FF4FA63428AA0
:107850009A4202D2521C428200E04382874A92F846
:107860002220802A0CD302F03F020A70B1F90620D0
:10787000402A06DBFF2A04D0C2883AB1521EC280D9
:10788000F0BDBDE8F0407B48FFF788BD428A9A42D0
:10789000F6D307784FF0010E3A074FF0FF055BD59E
:1078A000847A40F2DC52630708D444F00403837204
:1078B000C28081F80BE081F80AE04CE04378072BA6
:1078C00005D0032B03D0052B01D0062B07D166066C
:1078D00005D444F040038372C280052239E0654A32
:1078E0005FEA437C02F138024FF42076127A0DD51C
:1078F0005FEAC26C0AD45FEA446C07D442F010021B
:1079000002723A0628D4C680192222E0DF0709D085
:10791000970707D4670605D442F002020272C680B8
:10792000042216E09F0709D5170707D4670605D478
:1079300042F008020272C68003220AE01B070BD540
:10794000530709D4630607D442F004020272C680CA
:107950000B22CA728A72CD80494AB2F92230B2F93A
:107960001A7003F23D140022A74200DB0276414E5A
:10797000444C06F13806A479B6895FEAC46C06F176
:1079800001064FF4C874B6B213D58681B6F57A7F76
:1079900005D9017A21F0800101728281F0BD037A5C
:1079A0001E06FBD4828143F080020272C480112043
:1079B00035E09F4216DA037E052B13D28681B6F599
:1079C000487F04D98281027A22F040020272027A50
:1079D0005606E3D45B1C037642F040020272C48078
:1079E00002201CE0284B1C89C4F3C006C4F3002706
:1079F00040F2EE24BE4216D11E78360713D4427EE2
:107A0000012ACBD1428BB2F5167F02D2521C42839F
:107A1000F0BD827A42F002028272C4800F20C872E6
:107A20008872CD80F0BD93F80D714FF40046012FA0
:107A300018D1164F41F6583C7F6C674512DD83F82C
:107A40000CE1134B1E60C38AA34202D25B1CC382AB
:107A5000F0BD4FF4FA73C3801C23CB728B72CD80C0
:107A6000C282F0BDC2820A4883F80C21001F066062
:107A7000F0BD000098060020F8060020CC0500208C
:107A8000B4040020100A0020980200203C010020CD
:107A9000140801402DE9F05FFB48FC49DFF8F0A332
:107AA000007E0A1D131D0128504658D030F85A4F49
:107AB0000C8041881180BAF85E001880F54DF64CB4
:107AC00049F2CD32B5F91E006083B5F9201043F6B6
:107AD000CC4C00EB410151430914A183B4F922308D
:107AE000B4F9206001FB03F200FB062242F38F325F
:107AF0006282B4F9167007FB0CF7BF1340F2333CF7
:107B0000714302FB0CF200FB131007EBA232E2827E
:107B100040F38F30A082B4F91810E04FC1EBC101DF
:107B200041F3D10101EBE000DD4E2083786C306041
:107B3000316930468847DB49308948800846FDF77F
:107B40005BFFDFF8649301264FF0000B99F800000B
:107B500008280CD0618E218204284AD01AE030F81F
:107B6000604F0C8041881180BAF86400A5E7CF48C7
:107B700090F92F10491C022939D890F86C1019B1CE
:107B8000B4F85200208205E0618E2182A4F85210E0
:107B900080F86C60B4F91410B4F90A00C44AF9F71B
:107BA0007FFCE062BAF91611884204DDC048E16248
:107BB000027B91404162B848DFF8F8E24C3847F266
:107BC000A30802784EF2461172B3012A52D080F80F
:107BD00000B000BF99F8000004280DD0B44AB4F9F1
:107BE0001210B4F90800283AF9F75AFC07E0608E41
:107BF000C8E7686A0014E062B87A70B3AE48AF4D67
:107C0000A0622860E06A68602846FCF7C9F8A84FBF
:107C1000287C3C3F01285ED0A06A3860A8480178E3
:107C2000C9075CD040695BE0B5F91E2042448A4236
:107C300009D8B5F9202042448A4204D8B5F9222057
:107C400042448A42C6D9A0F802B0B7F8AE205946DD
:107C5000B2F5C87F02D8467007E039E0B2F5487F38
:107C600001D8022200E0032242708AF80F1089F83E
:107C7000001024E080F800B0B5F91EC05A46C44494
:107C80008C4509D8B5F920C0C4448C4504D8B5F951
:107C9000225045448D429DD9B7F8AE10B1F5C87F4A
:107CA00001D8467006E0B1F5487F01D8022100E016
:107CB0000321417042808AF80F2089F80020BEF825
:107CC000061041F40061AEF80610FAF76FF981E78B
:107CD0004FF4AF7093E768693860A86900E0E06A24
:107CE000786073483C38FCF7CFF96B4D6A4935F83A
:107CF000100F3C39FFF742FDDFF89C91DFF8C4819B
:107D0000A9F14C09D9F81010C9F86C10B5F9101088
:107D1000B868B5F9122000FB01F4FB68504303FB7F
:107D2000124444F38F3703FB010040F38F34AF86D6
:107D3000EC86A8F802704546A8F804404046FEF7D5
:107D400007FA287F09F11405012830D0604241105C
:107D50004DF6B35047433A1469802A808B18A9F82E
:107D60000440A9F80630891AA9F808108AF80CB05E
:107D7000B9F90430D84654464946002B00DD267335
:107D8000B1F90600002802DD227B921C2273B9F9AA
:107D90000820002A02DD217B091D2173217B072990
:107DA00020D2DFE801F01F1B3419301D3200B8F972
:107DB00020304DF6B352584240106880B8F91E107A
:107DC000514309142980A9F804304318A9F8063052
:107DD000401AA9F80800C9E7667303E0022100E031
:107DE00003216173DFF8B090374E384F99F80010D7
:107DF0000129617B0DD0072945D2DFE801F0E7FEBC
:107E0000FDFCFBFAF9000421EBE70521E9E7062177
:107E1000E7E7072937D2DFE801F0D9041B62799937
:107E2000AF0001461846FBF761FE2860B5F9020075
:107E3000B5F9001043F2046201445143090C504368
:107E4000A4F85A10000CA4F85C00A4F85E8027E1A6
:107E5000404201B2504200B2FBF748FE2860B5F93B
:107E6000020043F204614143090CA4F85A10B5F929
:107E70000010084443F204614843000CA4F85C007D
:107E8000A4F85E803AE1A1E090090020342C014082
:107E9000980200201C050020600000203C0100200A
:107EA00028040020E8030020EF060020240A002018
:107EB0008C080020100A0020A2FEFFFFE809002025
:107EC00008090020C40900200024014000280140C6
:107ED0003046F8F7CBFE01231A4607216BE019461E
:107EE0001046FBF703FE2860A4F85A80B5F902009B
:107EF000B5F9001043F2046201445143090C5043A8
:107F0000A4F85C10000CA4F85E0026E1594240423F
:107F100009B200B2FBF7EAFD2860A4F85A80B5F96F
:107F2000020043F204614143090CA4F85C10B5F966
:107F30000010084443F204614843000C39E1304624
:107F4000F8F794FE01231A46052134E01146FBF7A9
:107F5000CDFD2860B5F9020043F204614143090CEC
:107F6000A4F85A10A4F85C80B5F90010084443F254
:107F700004614843000C47E1504201B2584200B24C
:107F8000FBF7B4FD2860B5F90200B5F9001043F223
:107F9000046201445143090CA4F85A105043A4F858
:107FA0005C80000CA4F85E005EE13046F8F75EFEEF
:107FB00001231A4606213846F8F758FE01213046BB
:107FC000F8F7CAFD01213846F8F7C6FDB34EB9F8F7
:107FD00008004D463080B9F80A007080B9F81000EA
:107FE000B0803046F9F798FCB4F85A00F18805E003
:107FF00018E1ECE0BDE08EE05EE031E00844A4F87A
:108000006000B4F85C0031890844A4F86200B4F858
:108010005E0071890844A4F86400317EA0480129FB
:1080200078D034F85A1F018061884180A18881800E
:108030009B49028808310A8042884A80808888806B
:108040009748896A0830884795F8360000287DD01F
:10805000F9F710F815F8360F401E2870BDE8F09FAC
:1080600001461846FBF742FD2860B5F9020040F6CC
:108070008151484380136880B5F9001040F6815261
:10808000514389134218A2F6815252425208298064
:10809000A4F85E201044A4F85C000844A4F85A0038
:1080A00000213046F8F758FD00213846F8F754FD16
:1080B00001231A4606210BE7404201B2504200B2AA
:1080C000FBF714FD2860B5F9020040F681514843E2
:1080D00080136880B5F9001040F68152514389132E
:1080E0004218A2F68152524252082980A4F85E201A
:1080F0001044A4F85A000844A4F85C00002130465B
:10810000F8F72AFD00213846F8F726FD01231A4624
:108110000521DDE6B4E019461046FBF7E7FC2860D0
:10812000B5F9020040F68151484380136880B5F9E3
:10813000001040F68152514389134218A2F6815231
:10814000524229805208A4F85A2000E09BE01044D3
:10815000A4F85E000844A4F85C0000213046F8F75B
:10816000FBFC00213846F8F7F7FC01231A460721EB
:10817000E5E65942404209B200B2FBF7B7FC28607D
:10818000B5F9020040F68151484380136880B5F983
:10819000001040F68152514389134218A2F68152D1
:1081A000524252082980A4F85A201044A4F85C00D6
:1081B0000844A4F85E0000213046F8F7CDFC002109
:1081C0003846F8F7C9FC01231A460621B7E61146DE
:1081D000FBF78CFC2860B5F9020040F6815148435A
:1081E00080136880B5F9001040F68152514389131D
:1081F0004218A2F68152524252082980A4F85C200B
:108200001044A4F85A000844A4F85E000021304647
:10821000F8F7A2FC00213846F8F79EFC01231A4625
:108220000521C2E6504201B2584200B2FBF75EFCA3
:108230002860B5F9020040F68151484380136880F8
:10824000B5F9001040F68152514389134218A2F645
:108250008152524252082980A4F85C201044A4F8AC
:108260005E000844A4F85A0000213046F8F774FC78
:1082700000213846F8F770FC01231A46072194E6DE
:1082800034F8601FCFE607480088A0F5D041683970
:108290003FF4E4AEBDE8F05FF9F7CEBD90090020F1
:1082A0002C000020182C01402DE9F041904C914801
:1082B000B4F85A100288511A89B20F296FD3008876
:1082C000A4F85A008C480088DFF83082C0074FF0CD
:1082D00000054FF0010741D0874AD4E90C10243241
:1082E0001388B1EB530F02D21288511A08444FF48D
:1082F000F371884200D208468149B1FBF0F0616C0D
:10830000C1F35101084406466064F8F788F800227A
:108310007C4BF7F7F0FF4FF040427B4BF7F7EBFF5A
:108320000E22F8F757F8F8F7B1F8A4F8A40094F87B
:108330006500401CC0B284F86500082834D36C483E
:1083400098F84620001F03789A4201D002704580B9
:108350006E4A13786E4A23B1458021E06564A564B6
:1083600058E0D8F89410A1F5FA618E4211DD616DE4
:108370008B1C9E4205DDB0F902100A290DDA491C5A
:1083800006E08E4205DAB0F90210002908DD491E28
:108390004180B0F902000A2802DB177001E0A2E078
:1083A0001570666584F865505A484FF4A542017807
:1083B000C1F38101012949D002294AD044F68771CD
:1083C0002181A4F8A020B0F9243089B24B439B133B
:1083D000A4F89C30B0F90E0000237043B0FBF1F01C
:1083E000A16CC0F3D100C1EBC101C90200EB913017
:1083F000A064F017810341EA9641B003F7F794FEB9
:10840000B4F8A210C1EBC101C902C00800EB913061
:10841000A4F8A200616CA06E0844A06694F86C20D9
:10842000521CD2B284F86C20082A05D3C008A4F8E4
:108430006E0084F86C50A566374A384ED3885806CB
:1084400033D498F80F00022806D02CE043F20451F0
:10845000B6E744F24621B3E7B06840F69916B04259
:1084600021DD94F8380094F88660B0420CD084F88E
:10847000860094F83D0000F00106C0F340008642FB
:1084800002D1A4F8825004E0B4F88200B0F5966FEF
:1084900005D2B4F88200401CA4F8820005E043F045
:1084A0008000D08001E0A4F88250114894F83F2069
:1084B000B0300C2A01D2C57400E0C774174B41F2EA
:1084C000482641F2504C93F83C400C4B0C2AB3F830
:1084D00082300AD3B14208DB012C06D0614502DDAF
:1084E000002B00D18774BDE8F0818574FBE70000A4
:1084F0003C010020F8060020000400409802002003
:108500004564BD0100209C40133B3340E60300203E
:10851000E7030020B4040020100A00201C050020FE
:108520002DE9F041384C394E394F207841F2333142
:10853000C2074FF000050CD0A28962B394F907007E
:10854000002800DA4042C0B2032829D240F2AE70BF
:108550002AE0A570E5732F4AE571A58192F83830BD
:10856000237220F00800A18040F0020020703D86B8
:108570007560B560F560916C490005D041F6846185
:10858000A18140F010002070C0B240F001002070C6
:108590006574BDE8F081658120F01000207015E061
:1085A000042803D240F6510060810FE0052802D272
:1085B00040F69910F8E740F6CC42062803D3072886
:1085C00001D3082801D2628100E0618197F89D0003
:1085D00098B9B088102301B2B4F90A003622FCF72A
:1085E00087F97060F168401AB1680844B060B6F964
:1085F00000104843C013F0603886388E10B1012057
:10860000A070C6E7A570C4E71C0C00207806002007
:10861000980200203C0100202DE9F041554C2678BD
:10862000F0077CD05448217A544D90F838008142AC
:108630007BD0534A2346DFF84CC1575C93F90E2098
:1086400093F90730874203D01CF80170874213D199
:1086500046F002065B1C26705BB2E3711CF8011049
:10866000814201D15B1CE37194F90710062901DDF9
:108670000621E171521C1CE0434F17F801C0434F23
:10868000844503D017F801C0844513D126F00206B3
:108690005B1E26705BB2E371795C814201D15B1E87
:1086A000E37194F907306FF005018B4200DAE17154
:1086B000521EA273207294F907108A1C042A02D950
:1086C00041F68462A2812C4A012912780ADD2B4BE3
:1086D00056079B6802D543F0080301E023F0080326
:1086E000AB606070B1F1FF3F09DA5107A96802D5AC
:1086F00021F0080101E041F00801A9606070F9F77C
:108700003FFEA078012810D121488068A3280CDA08
:1087100094F90700022803DD0220E07105E01EE065
:108720006FF00101884200DAE171A089002630B1C2
:10873000401E0004000CA08101D1E671A673E87B05
:1087400004280CD0B5F93010512341220020FCF749
:10875000CFF82886002802D1E07B10B1A670BDE8D2
:10876000F0810C4806700C480670207820F001005B
:108770002070F4E71C0C00203C010020980200202F
:10878000B8930008BE930008CA930008D09300086D
:108790001C0500200C070020EF060020743F713DEF
:1087A0009B3BED396238F436A13565343F332A32CC
:1087B000273133304C2F722EA32DDF2C242C722B1B
:1087C000000000361C070038AA0A003AAA0A003C3A
:1087D000CC0C003ECC0C0040380E0042380E004459
:1087E000380E0046380E0048380E004AC711004CBB
:1087F000C711004EC7110050C7110052C7110054D5
:10880000C7110056C7110058C711005AC711005CA4
:10881000C711005EC7110060C7110062C711006474
:10882000C7110066C7110068C711006A0000003652
:10883000000000388E03003A8E03003CFA04003E2C
:10884000FA0400401C0700421C0700441C070046B5
:108850001C0700481C07004A8808004C8808004E86
:10886000880800508808005288080054880800567C
:10887000880800588808005A8808005C8808005E4C
:10888000880800608808006288080064880800661C
:10889000880800688808006A000000360000003878
:1088A0008E03003A8E03003CFA04003EFA040040B6
:1088B0001C0700421C0700441C0700461C07004818
:1088C0001C07004A8808004C8808004E88080050A1
:1088D0008808005288080054880800568808005804
:1088E0008808005A8808005C8808005E88080060D4
:1088F00088080062880800648808006688080068A4
:108900008808006A0000003A2202003C8E03003E04
:10891000B0050040D2070042AA0A0044CC0C004631
:10892000EE0E00481111004A3313004C9F14004E04
:108930000B16005077170052771700547717005620
:10894000771700587717005A7717005C7717005E83
:108950007717006077170062771700647717006653
:10896000771700687717006A7717006C7717006E23
:1089700000000036000000388E03003A8E03003CF1
:10898000FA04003EFA0400401C0700421C070044A1
:108990001C0700461C0700481C07004A8808004CBA
:1089A0008808004E88080050880800528808005443
:1089B00088080056880800588808005A8808005C13
:1089C0008808005E880800608808006288080064E3
:1089D00088080066880800688808006A0000003A75
:1089E0002202003C4404003E660600408808004223
:1089F000AA0A0044CC0C0046EE0E00481111004AB1
:108A00003313004C9F14004E0B1600507717005282
:108A1000E31800544F1A0056BB1B0058271D005A7C
:108A2000DD1D005C931E005E491F00600020006297
:108A3000B52000646C21006622220068D822006AFA
:108A40008E23006C4424006E0000003400000036C9
:108A5000000000380000003A0000003C0000003E2A
:108A600000000040000000420000004400000046FA
:108A7000000000480000004A0000004C0000004ECA
:108A8000000000500000005200000054000000569A
:108A9000000000580000005A0000005C0000005E6A
:108AA000000000600000006200000064000000663A
:108AB00000000068441458585870111158585870E4
:108AC000411158584870111448585870141158489A
:108AD00058703313005695130054B61300525A14AD
:108AE0000050FD14004EA115004C4516004A7616A4
:108AF00000486C17004672180044BA190042741BF3
:108B00000040911D003EB420003C9F22003AE1222B
:108B10000038532300368B240034812500322B2764
:108B200000302028002E5829002CB02A002A9B2C27
:108B30000028D22D00267C2F00242631002202336B
:108B40000020FD34001E5C37001CCC3C001A873E20
:108B50000018BE3F00160040001400400012004004
:108B600000100040000E0040000C0040000A0040D1
:108B700000080040000600400004004000020040E1
:108B800000000000010203040500050001020304C7
:108B90000104000305020000F0010000360100009E
:108BA000F8000000BA0000007C0000007C0000001B
:108BB0007C000000411414111114441114144111CB
:108BC0000000290052007B00A400CC00F5001E012B
:108BD000470170019901C201EA0113023C026502DA
:108BE0008E02B602DF020803300359038203AA0390
:108BF000D303FB0324044C0475049D04C504EE0454
:108C000016053E0567058F05B705DF0507062F0624
:108C100057067F06A706CE06F6061E0746076D070F
:108C20009507BC07E4070B08320859088108A80813
:108C3000CF08F6081D0944096A099109B809DE0937
:108C4000050A2B0A520A780A9E0AC40AEA0A100B7D
:108C5000360B5C0B820BA80BCD0BF30B180C3E0CE8
:108C6000630C880CAD0CD20CF70C1C0D410D650D7E
:108C70008A0DAF0DD30DF70D1C0E400E640E880E3D
:108C8000AC0ECF0EF30E170F3A0F5E0F810FA40F2D
:108C9000C70FEA0F0D103010531075109810BA104E
:108CA000DD10FF102111431165118711A911CA119F
:108CB000EC110D122E12501271129212B312D41224
:108CC000F41215133613561376139613B713D713DE
:108CD000F61316143614561475149414B414D314CD
:108CE000F214111530154E156D158C15AA15C815F1
:108CF000E7150516231641165F167C169A16B71649
:108D0000D516F2160F172C17491766178317A017D9
:108D1000BC17D917F51711182E184A18661881189C
:108D20009D18B918D418F0180B19261942195D1995
:108D300078199219AD19C819E219FD19171A311AC3
:108D40004C1A661A801A991AB31ACD1AE61A001B21
:108D5000191B331B4C1B651B7E1B971BAF1BC81BB2
:108D6000E11BF91B121C2A1C421C5A1C721C8A1C77
:108D7000A21CBA1CD21CE91C011D181D301D471D68
:108D80005E1D751D8C1DA31DBA1DD01DE71DFD1D8B
:108D9000141E2A1E401E571E6D1E831E981EAE1ED8
:108DA000C41EDA1EEF1E051F1A1F2F1F451F5A1F54
:108DB0006F1F841F991FAE1FC21FD71FEC1F0020FB
:108DC00000006400C9002D019201F7015B02C0029E
:108DD00024038903ED035204B6041A057F05E30555
:108DE0004706AB060F077307D7073B089F08020922
:108DF0006609C9092D0A900AF30A560BB90B1C0C17
:108E00007F0CE20C440DA60D090E6B0ECD0E2F0F3C
:108E1000900FF20F5310B41015117611D7113812AC
:108E20009812F8125813B81318147714D61435156D
:108E30009415F3155116B0160E176B17C91726188F
:108E40008318E0183D199919F519511AAD1A081B24
:108E5000631BBE1B181C731CCD1C261D801DD91D39
:108E6000321E8A1EE31E3B1F921FEA1F41209820DC
:108E7000EE2044219A21EF2145229922EE2242231D
:108E80009623E9233C248F24E22434258525D72505
:108E900028267826C82618276827B72706285428A2
:108EA000A228EF283D298929D629222A6D2AB82A05
:108EB000032B4D2B972BE12B2A2C722CBB2C022D34
:108EC0004A2D912DD72D1D2E632EA82EEC2E302F3E
:108ED000742FB82FFA2F3D307F30C030013141312F
:108EE0008131C13100323F327D32BA32F732343310
:108EF0007033AC33E73322345C349534CE340735E9
:108F00003F357735AE35E4351A3650368536B936C5
:108F1000ED36203753378637B737E93719384938B0
:108F20007938A838D738053932395F398B39B739AC
:108F3000E2390D3A373A603A893AB23ADA3A013BC5
:108F4000283B4E3B733B983BBD3BE03B043C263CFF
:108F5000483C6A3C8B3CAB3CCB3CEA3C093D273D62
:108F6000443D613D7D3D993DB43DCE3DE83D013EF2
:108F70001A3E323E493E603E763E8C3EA13EB53EB4
:108F8000C93EDC3EEF3E013F123F233F333F433FAC
:108F9000513F603F6E3F7B3F873F933F9E3FA93FDE
:108FA000B33FBC3FC53FCD3FD53FDC3FE23FE83F4D
:108FB000ED3FF13FF53FF93FFB3FFD3FFF3FFF3FF7
:108FC000FF3F0000E7382C35002020EF203720231A
:108FD0003320262021000080020004000800100039
:108FE0000002000400080400000200040008001051
:108FF00000200040008004000000008000000040CD
:109000000000002000000010000000080000000424
:10901000000000020000000100008000000040008D
:109020000000200000001000000008000000040004
:109030000000020000000100008000000008014064
:10904000000C0140000C0140000C0140000C0140EC
:10905000000C0140000C0140000C014000100140D8
:1090600000100140001001400010014000100140BC
:1090700000100140001001400010014000140140A8
:1090800004080140040C0140040C0140040C0140A0
:10909000040C0140040C0140040C0140040C01408C
:1090A000041001400410014004100140041001406C
:1090B000041001400410014004100140041001405C
:1090C0000414014008080140080C0140080C01404C
:1090D000080C0140080C0140080C0140080C01403C
:1090E000080C014008100140081001400810014020
:1090F000081001400810014008100140081001400C
:1091000008100140081401400C0801400C0C0140FB
:109110000C0C01400C0C01400C0C01400C0C0140EB
:109120000C0C01400C0C01400C1001400C100140D3
:109130000C1001400C1001400C1001400C100140BB
:109140000C1001400C1001400C14014010080140AB
:10915000100C0140100C0140100C0140100C01409B
:10916000100C0140100C0140100C01401010014087
:10917000101001401010014010100140101001406B
:109180001010014010100140101001401014014057
:1091900000000000000000000000000000000000CF
:1091A0000000000014080140140C0140140C0140A0
:1091B000140C0140140C0140140C0140140C01402B
:1091C000140C01401410014014100140141001400F
:1091D00014100140141001401410014014100140FB
:1091E00014100140141401400000000000000000B1
:1091F000000000000000000000000000FFFFFF0F63
:109200000FFFFFFFFFF0FFFFFF0FFFFFFFFFF0FF6C
:109210000FFFFFFFFFF0FFFFFF0FFFFFFFF0FFFF5C
:109220000FFFFFFFFFF0FFFFFF0FFFFFFFFFF0FF4C
:10923000FFFF0FFFFFFFFFF0FFFFFF0FFFF0FFFF3C
:10924000000000404000000000040000004000005A
:109250000000040040000000000400000040000086
:109260000004000040000000000400000040000076
:109270000000040000004000000000040000004066
:1092800000040000000000808000000000080000D2
:1092900000800000000008008000000000080000BE
:1092A00000800000000800008000000000080000AE
:1092B000008000000000080000008000000000089E
:1092C00000000080000800000000002020000000D6
:1092D000000200000020000000000200200000004A
:1092E000000200000020000000020000200000003A
:1092F000000200000020000000000200000020002A
:1093000000000002000000200002000000000060D9
:109310006000000000060000006000000000060081
:109320006000000000060000006000000006000071
:109330006000000000060000006000000000060061
:109340000000600000000006000000600006000051
:109350000080020004000800100000020004000861
:1093600004000002000400080010002000400080FB
:1093700004000000FF7FFFFFFDFFFFFFFBFFFFFF7B
:10938000F7FFFFFFEFFFFFFFFFFDFFFFFFFBFFFF0B
:10939000FFF7FFFFFBFFFFFFFFFDFFFFFFFBFFFFEF
:1093A000FFF7FFFFFFEFFFFFFFDFFFFFFFBFFFFF45
:1093B000FF7FFFFFFBFFFFFF010203040500020325
:1093C0000405000103040500010205000102030475
:1093D00004050001020355050010AA1A55250030A6
:1093E000AA3A0000AA0A55150020AA2A5535FF3FBF
:1093F000109400080000002020070000E806000884
:109400000095000820070020C0090000246400081F
:1094100045020406082D010203040405440607085A
:109420000913C52B1B08D904211355152A40061909
:1094300008019713E53D1408093E1B080504012D9A
:1094400017020604050103148020FF8BAA0A0201FB
:109450009C15AA0A551500085920AA2A5535FF3F20
:10946000072903010504060203127C1573FFFF049C
:10947000FF8080010125025B6402130A13916712C9
:10948000081201100C05040602030101030705057B
:10949000280B010203040206070303040C3D070620
:1094A000040509191F191904310506064BAA1A02E9
:1094B0004B381E026910312E40FD39692602110415
:1094C0002F405F020C26405B262ACD5515551512FC
:1094D0003902017F0316D0071AFF01013B0261AA7E
:1094E0006C080108A80916C491220312100A17403B
:1094F0001C12600A16901B014913A56702000800A0
:020000040800F2
:10FC00004A46545A594D46312D4E3330202020203B
:10FC1000050406020301AA0AAA0AAA0AAA0AAA0A4B
:10FC2000AA0ADE3F00100000FF0131000201664613
:10FC300000400040513800400040004000400101B9
:10FC400000400040FF387B257B257B25FF003333B8
:10FC50000201401F00016626B81E6626FFFFFFFF57
:10FC6000FFFF01010100010000000300000200008D
:04FC70000000AA5591
:04000005080000ED02
:00000001FF
